:10000000A2C20000D1C20000CFC20000CDC20000D9
:10001000CBC20000C9C20000C7C20000C5C20000B8
:10002000C3C20000C1C20000BFC20000BDC20000C8
:10003000BBC20000B9C20000B7C20000B5C20000D8
:10004000B3C200000C94B610AFC20000ADC20000F5
:100050000C94E310A9C20000A7C200000C94620F28
:10006000A3C200000C94750D0C944C0D9DC20000B1
:100070009BC2000099C2000097C2000095C2000018
:100080000C94891091C200008FC200008DC2000044
:100090008BC2000089C2000087C2000085C2000038
:1000A00083C2000081C200000C945C107DC200007D
:1000B0007BC2000079C2000077C200000C942F10B0
:1000C00073C2000071C200006FC200006DC2000068
:1000D0006BC2000069C2000067C2000065C2000078
:1000E00063C20000E002ED02F602FF020C031503FA
:1000F0009606960696069606960622032F033C035E
:100100009606490352035B03680371037A03830372
:100110008C03950396069E03A703B00396069606E6
:100120009606B903C203CB0396069606D403E103F1
:10013000960696069606EE03FB030804960615043B
:100140001E042704960696069606300439044204D7
:1001500096064F045C046904960696069606760495
:100160008304900496069D04AA04B7049606960696
:100170009606C404D104DE049606960696069606F4
:10018000960696069606960696069606960696068F
:10019000960696069606960696069606960696067F
:1001A0009606960696069606960696069606060500
:1001B0000F051805960621052A05330596069606AD
:1001C00096063C05490556059606630570057D05AE
:1001D0009606960696068A059705A4059606B10525
:1001E000BA05C305960696069606CC05D505DE0526
:1001F000960696069606960696069606960696061F
:10020000960696069606EB04F404FD0496069606FA
:1002100096069606960696069606960696069606FE
:1002200096069606960696069606960696069606EE
:1002300096069606960696069606960696069606DE
:1002400096069606960696069606960696069606CE
:1002500096069606960696069606960696069606BE
:1002600096069606960696069606960696069606AE
:10027000960696069606E705F005FD0596060A061B
:10028000130620069606960696062D0636064306A3
:100290009606500659066606960696069606730654
:1002A0007C0689064F0B520B410B450B4B0B890B00
:1002B000560B5A0B600B640B680B6E0B720B760BB4
:1002C000890B7C0B800B840BB517BA17BF17C917A6
:1002D000D3174C18DD17E517ED17F71701180B1892
:1002E0001A1824184C182E183818421800000A0B37
:1002F00002090C0D0E0807030401000000000000B5
:1003000000000000000000000000000000000000ED
:1003100000000000000000001211100000000000AA
:1003200000000000000000000000000000000000CD
:10033000000000002100240027002A002D003000CA
:10034000330001010000040107010A01000022003E
:10035000250028002B002E0031003400020100008F
:10036000050108010B0100002000230026002900E0
:100370002C002F00320000010000030106010901DA
:1003800005050505070508080808020202020A0A11
:10039000080804040404010101010101010103032F
:1003A000030303030303040707070C0C0C0C0C0CDA
:1003B0000C0C0202020206060606060606060B0BD7
:1003C0000B0B0B0B0B0B0102102020080810204018
:1003D0001020408002010201080402010102040809
:1003E0001020408080402010080402018004020197
:1003F00080402010080402010804020101020408E0
:100400001020408001020408102040804E414E49D7
:100410004E495459494E46CDCCCC3D0AD7233C17C2
:10042000B7D13877CC2B329595E6241FB14F0A000F
:100430000020410000C84200401C4620BCBE4CCAFF
:100440001B0E5AAEC59D7400407A10F35A00A0727C
:100450004E18090010A5D4E80000E87648170000FF
:10046000E40B54020000CA9A3B000000E1F50500CD
:100470000080969800000040420F000000A0860116
:10048000000000102700000000E8030000000064E6
:1004900000000000000A0000000000010000000051
:1004A000002C76D888DC674F0823DFC1DFAE59E126
:1004B000B1B796E5E3E453C63AE651997696E8E695
:1004C000C28426EB898C9B62ED407C6FFCEFBC9C68
:1004D0009F40F2BAA56FA5F490055A2AF75C936B7A
:1004E0006CF9676DC11BFCE0E40D47FEF520E6B535
:1004F00000D0ED902E0300943577050080841E080F
:100500000000204E0A000000C80C333333330F982C
:100510006E12831141EF8D2114893BE65516CFFEF3
:10052000E6DB18D1844B381BF77C1D901DA4BBE47F
:1005300024203284725E228100C9F124ECA1E53DC1
:100540002700CE44C94411241FBECFEFD1E2DEBF45
:10055000CDBF00E00CBF17E0A0E0B2E0E6EBFDE9A4
:1005600000E00BBF02C007900D92A432B107D9F78B
:100570002CE0A4E2B7E001C01D92AE3CB207E1F767
:1005800012E0C2EAD2E000E006C021970109802F04
:10059000FE010E945545C13AD10780E00807A9F73E
:1005A0000E94EF3A0C94C94E2BCD603E710508F0C5
:1005B000BDC3FB018827EE58FF4F8F4F0C94554564
:1005C00081E090E0A0E0B0E08093280790932907B5
:1005D000A0932A07B0932B07089510922C0710922E
:1005E0002D0710922E0710922F07089510923007B2
:1005F000109231071092320710923307089581E06C
:1006000090E0A0E0B0E08093340790933507A0938A
:100610003607B093370708951092380710923907BC
:1006200010923A0710923B07089583E090E0A0E013
:10063000B0E080933C0790933D07A0933E07B093B2
:100640003F07089588E790E0A0E0B0E0809354076A
:1006500090935507A0935607B0935707089588E7DE
:1006600090E0A0E0B0E08093580790935907A093E2
:100670005A07B0935B07089588E790E0A0E0B0E0E8
:1006800080935C0790935D07A0935E07B0935F072C
:1006900008951092640710926507109266071092F1
:1006A00067070895109268071092690710926A0709
:1006B00010926B07089581E090E0A0E0B0E0809395
:1006C0006C0790936D07A0936E07B0936F07089522
:1006D00010927007109271071092720710927307B0
:1006E0000895109274071092750710927607109271
:1006F00077070895109278071092790710927A0779
:1007000010927B07089510927C0710927D0710923B
:100710007E0710927F07089510928007109281073C
:100720001092820710928307089510928407109206
:1007300085071092860710928707089510928C07FC
:1007400010928D0710928E0710928F0708951092C5
:1007500090071092910710929207109293070895B4
:10076000109294071092950710929607109297078F
:1007700008951092A4071092A5071092A607109250
:10078000A70708951092A8071092A9071092AA0728
:100790001092AB0708951092AC071092AD0710921B
:1007A000AE071092AF07089581E090E0A0E0B0E0BE
:1007B0008093B8079093B907A093BA07B093BB078B
:1007C000089581E090E0A0E0B0E08093BC079093B2
:1007D000BD07A093BE07B093BF0708958CE291E0D8
:1007E000A0E0B0E08093CC079093CD07A093CE0714
:1007F000B093CF0708958CE291E0A0E0B0E0809341
:10080000D0079093D107A093D207B093D307089550
:100810008CE291E0A0E0B0E08093D4079093D507FC
:10082000A093D607B093D70708951092DC071092D3
:10083000DD071092DE071092DF0708951092E0079F
:100840001092E1071092E2071092E30708951092C8
:10085000E4071092E5071092E6071092E707089563
:100860001092F4071092F5071092F6071092F7070E
:1008700008951092F8071092F9071092FA07109253
:10088000FB07089581E090E0A0E0B0E08093FC07D2
:100890009093FD07A093FE07B093FF07089585E0AE
:1008A00090E0A0E0B0E08093040890930508A09346
:1008B0000608B0930708089585E090E0A0E0B0E056
:1008C0008093080890930908A0930A08B0930B0836
:1008D000089589E190E0A0E0B0E080930C08909347
:1008E0000D08A0930E08B0930F08089582E390E0DE
:1008F000A0E0B0E080931C0890931D08A0931E0810
:10090000B0931F08089582E390E0A0E0B0E08093E8
:10091000200890932108A0932208B09323080895FB
:1009200082E390E0A0E0B0E0809324089093250853
:10093000A0932608B0932708089582E390E0A0E0F2
:10094000B0E080932C0890932D08A0932E08B093CC
:100950002F08089582E390E0A0E0B0E08093300893
:1009600090933108A0933208B0933308089582E33E
:1009700090E0A0E0B0E08093340890933508A09315
:100980003608B0933708089580E991E0A0E0B0E020
:100990008093440890934508A0934608B093470875
:1009A000089580E991E0A0E0B0E08093480890933A
:1009B0004908A0934A08B0934B08089580E991E054
:1009C000A0E0B0E080934C0890934D08A0934E08AF
:1009D000B0934F08089510926C0910926D0910920F
:1009E0006E0910926F0908951092700910927109A2
:1009F000109272091092730908951092740910925E
:100A00007509109276091092770908951092BC0822
:100A10001092BD081092BE081092BF08089510925F
:100A2000C0081092C1081092C2081092C30808951D
:100A30001092C4081092C5081092C6081092C708F8
:100A400008951092CC081092CD081092CE08109202
:100A5000CF0808951092D0081092D1081092D208B1
:100A60001092D30808951092D4081092D5081092CD
:100A7000D6081092D708089585E090E0A0E0B0E095
:100A80008093E4089093E508A093E608B093E70804
:100A9000089585E090E0A0E0B0E08093E8089093AE
:100AA000E908A093EA08B093EB08089585E090E088
:100AB000A0E0B0E08093EC089093ED08A093EE08DE
:100AC000B093EF08089584EB95E1A0E0B0E0809347
:100AD000F4089093F508A093F608B093F7080895EA
:100AE00084EB95E1A0E0B0E08093F8089093F908DA
:100AF000A093FA08B093FB08089584EB95E1A0E079
:100B0000B0E08093FC089093FD08A093FE08B0939A
:100B1000FF08089585E090E0A0E0B0E080930C0924
:100B200090930D09A0930E09B0930F09089585E0E5
:100B300090E0A0E0B0E08093100990931109A09399
:100B40001209B0931309089585E090E0A0E0B0E0A9
:100B50008093140990931509A0931609B09317096F
:100B6000089510921C0910921D0910921E091092EE
:100B70001F0908951092200910922109109222094C
:100B800010922309089510922409109225091092B9
:100B900026091092270908951092340910923509F8
:100BA0001092360910923709089510923809109260
:100BB000390910923A0910923B09089510923C09A4
:100BC00010923D0910923E0910923F09089510922B
:100BD0004C0A10924D0A10924E0A10924F0A089534
:100BE0008CE390E0A0E0B0E08093500A9093510A2B
:100BF000A093520AB093530A089581E090E0A0E0D8
:100C0000B0E08093540A9093550AA093560AB0938B
:100C1000570A089510925C0A10925D0A10925E0ABB
:100C200010925F0A08958CE390E0A0E0B0E080931A
:100C3000600A9093610AA093620AB093630A0895D0
:100C400081E090E0A0E0B0E08093640A9093650AB0
:100C5000A093660AB093670A08951092740A1092DE
:100C6000750A1092760A1092770A08958CE390E044
:100C7000A0E0B0E08093780A9093790AA0937A0A72
:100C8000B0937B0A089581E090E0A0E0B0E080930B
:100C90007C0A90937D0AA0937E0AB0937F0A089500
:100CA0001092840A1092850A1092860A1092870A7E
:100CB00008958CE390E0A0E0B0E08093880A9093E0
:100CC000890AA0938A0AB0938B0A089581E090E084
:100CD000A0E0B0E080938C0A90938D0AA0938E0AD6
:100CE000B0938F0A089510929C0A10929D0A109258
:100CF0009E0A10929F0A08958CE390E0A0E0B0E075
:100D00008093A00A9093A10AA093A20AB093A30A89
:100D1000089581E090E0A0E0B0E08093A40A909371
:100D2000A50AA093A60AB093A70A0895660F771F95
:100D3000660F771FFB01E85DF84F10821182128267
:100D4000138208958FEF9FEF08958F929F92AF9235
:100D5000BF92CF92DF92EF92FF921F93CF93DF93D8
:100D60005B01EB01CC0FDD1FCE010E94564E182F08
:100D7000CE0101960E94564EC82ED12CE12CF12CAA
:100D80008DE8A81AB10883E0A816B10488F4CE0152
:100D900044960E94564E882E912CA12CB12CCE0147
:100DA00045960E94564E482F50E060E070E006C025
:100DB00040E050E0BA01812C912C5401FE2CED2C26
:100DC000DC2CCC24C10ED11CE11CF11C5401992453
:100DD00088248C0C9D1CAE1CBF1C742F66275527C5
:100DE0004427CB01BA01680D791D8A1D9B1DDF9137
:100DF000CF911F91FF90EF90DF90CF90BF90AF9079
:100E00009F908F9008958FE794E00E94A83981E128
:100E100093E00E94A8390E94EB240E94F52380E011
:100E200090E008950C9428480C9428480C94284885
:100E30000C9428480C9428480C9428480C94284872
:100E40000C9428480C9428480C9428484F925F92A0
:100E50006F927F928F929F92AF92BF92CF92DF92CA
:100E6000EF92FF920F931F93CF93DF9300D01F92C7
:100E7000CDB7DEB7FB011689078982889388A684DF
:100E8000B784C284D384E484F58446805780608428
:100E90007184428153816481758149835A836B8354
:100EA0007C830E9490161F921F921F920F931F9394
:100EB0009301820149815A816B817C810E9457197B
:100EC0000F900F900F900F900F9080E090E00F9098
:100ED0000F900F900F90DF91CF911F910F91FF9086
:100EE000EF90DF90CF90BF90AF909F908F907F90CA
:100EF0006F905F904F900895CF93DF93EB0120E0C8
:100F000030E040E85FE36A817B818C819D810E94B3
:100F10003A4D811113C084E894E00E94A8390E94E0
:100F20009016FC01E35BFF4F108211821282138244
:100F3000E25DFE4F108A118A128A138A20E030E0A7
:100F400040E85FE36E817F81888599850E943A4DF4
:100F5000811113C084E994E00E94A8390E94901680
:100F6000FC01EA53FF4F1082118212821382E15377
:100F7000FF4F108A118A128A138A20E030E040E87D
:100F80005FE36A857B858C859D850E943A4D811142
:100F900013C084EA94E00E94A8390E949016FC01D4
:100FA000E15CFE4F1082118212821382E059FF4FE2
:100FB000108A118A128A138A0E94EB240E94F52358
:100FC00080E090E0DF91CF9108950E94EB240E9491
:100FD000482480E090E0089584EB94E00E94A839D2
:100FE0000E94EB240E9452250E94EB240E940724B9
:100FF0000E94591840E050E068E070E00E94051738
:101000000E94591840E050E069E070E00E94051726
:101010000E94591840E050E06AE070E00E94051715
:101020000E94591840E050E06DE070E00E94051702
:1010300080E090E008950F931F93CF93DF93FB011F
:10104000C2A1D3A1068D178D8091680B9091690B79
:10105000892B41F481E090E00E9493479093690BC3
:101060008093680B0430110539F00530110541F407
:10107000BE0183EC9CE003C0BE0180EC9CE06CD719
:1010800080E090E0DF91CF911F910F910895EF9252
:10109000FF920F931F93CF93DF9300D01F92CDB792
:1010A000DEB78B017B01EE0CFF1C622FC701298389
:1010B0003A834B835C830E945E4E29813A814B8147
:1010C0005C81992757FD9A95852F742F632FC7014F
:1010D00001960E945E4E0D58110929813A814B817B
:1010E0005C8103301105A8F4BA01992777FD90952A
:1010F000892FC70144960E945E4E29813A814B8117
:101100005C81652F772788279927C70145960E941C
:101110005E4E80E090E00F900F900F900F90DF9167
:10112000CF911F910F91FF90EF900895CF92DF9292
:10113000EF92FF92CF93DF93EB010E94C1188823B7
:1011400059F1FE01EE0FFF1FEE0FFF1FE85DF84F94
:10115000C080D180E280F3808BEB94E00E94A839BC
:1011600082E894E00E94A8398FEB94E00E94A839AD
:10117000CE010E94EA3A82E894E00E94A83981EC0C
:1011800094E00E94A839C701B6010E94F4390E9478
:10119000EB240E94F52304C083EC94E00E94A8395C
:1011A00080E090E0DF91CF91FF90EF90DF90CF90C3
:1011B0000895EF92FF920F931F93CF93DF93809147
:1011C0006A0B90916B0B892B09F069C084E090E069
:1011D0000E949347EC0160E070E0B7DD1616170639
:1011E0008CF100E010E0B801CE010E94C118882304
:1011F00019F0B801CE01D9D90F5F1F4F013E11057B
:1012000091F798E2E92E97E0F92E00E010E0B8019E
:10121000CE010E94C118882341F0F701208131815D
:1012200042815381B801CE0132DF0F5F1F4FF4E0DE
:10123000EF0EF11C0639110551F7D0936B0BC093DB
:101240006A0B2DC088E2E82E87E0F82E00E010E05F
:10125000B801CE010E94C1188823C1F0B801CE01A7
:1012600074DDF70160837183828393836F3F7F4FC7
:101270008F4F9F4F59F4B801CE0197D9F7012081C4
:10128000318142815381B801CE0101DF0F5F1F4FD1
:10129000F4E0EF0EF11C013E1105D1F6CECF8091A6
:1012A0006A0B90916B0BDF91CF911F910F91FF9083
:1012B000EF9008954F925F926F927F928F929F92DC
:1012C000AF92BF92CF92DF92EF92FF920F931F9354
:1012D000CF93DF9300D01F92CDB7DEB76ADF409087
:1012E000040850900508609006087090070861DFB8
:1012F0008090080890900908A0900A08B0900B0808
:101300000E94EB24C090B00AD090B10AE090B20ADB
:10131000F090B30A0E94EB24C701B6010E94404D31
:101320006B017C01C301B2010E94404D9B01AC01E5
:10133000C701B6010E94C9452B013C016091B40A66
:101340007091B50A8091B60A9091B70A0E94404DFB
:101350006B017C01C501B4010E94404D9B01AC01B1
:10136000C701B6010E94C945AB01BC0149835A833C
:101370006B837C830E9490161F921F921F921F9274
:101380001F92812C912CA12CB12CC12CD12C760137
:1013900049815A816B817C818A019B01B301A20141
:1013A0000E9457190E9490161F921F921F921F921F
:1013B0001F9297018601B301A2010E9457190E9452
:1013C00090161F921F921F921F921F9297018601E3
:1013D000B701A6010E9457190FB6F894DEBF0FBEE1
:1013E000CDBF80E090E00F900F900F900F90DF91B5
:1013F000CF911F910F91FF90EF90DF90CF90BF9012
:10140000AF909F908F907F906F905F904F900895D6
:1014100008950895089508950895089508950895E4
:1014200008950895CF92DF92EF92FF920F931F934A
:10143000CF93DF936C017A018B01C0E0D0E0CE1531
:10144000DF0589F0D8016D918D01D601ED91FC91F8
:101450000190F081E02DC6011995892B11F47E01D0
:1014600002C02196ECCFC701DF91CF911F910F9160
:10147000FF90EF90DF90CF900895FC01918D828DC9
:10148000981761F0828DDF01A80FB11D5D968C91D8
:10149000928D9F5F9F73928F90E008958FEF9FEFE3
:1014A0000895FC01918D828D981731F0828DE80F9F
:1014B000F11D858D90E008958FEF9FEF0895FC0159
:1014C000918D228D892F90E0805C9F4F821B910926
:1014D0008F73992708958AE89BE0F1DF21E0892B3B
:1014E00009F420E0822F0895FC01848DDF01A80F0C
:1014F000B11DA35ABF4F2C91848D90E001968F733C
:101500009927848FA689B7892C93A089B1898C915A
:1015100080648C93938D848D981306C00288F38920
:10152000E02D80818F7D80830895EF92FF920F934D
:101530001F93CF93DF93EC0181E0888F9B8D8C8D7F
:10154000981305C0E889F989808185FD23C0F62EAE
:101550000B8D10E00F5F1F4F0F731127E02E8C8D46
:10156000E8120BC00FB607FCFACFE889F989808131
:1015700085FFF5CFCE01B8DFF2CF8B8DFE01E80FEE
:10158000F11DE35AFF4FF0820B8FEA89FB898081BE
:10159000806207C0EE89FF896083E889F9898081CC
:1015A0008064808381E090E0DF91CF911F910F9163
:1015B000FF90EF900895CF93DF93EC01888D8823FF
:1015C000C1F0EA89FB89808185FD05C0A889B989B8
:1015D0008C9186FD0EC00FB607FCF5CF808185FF8C
:1015E000F2CFA889B9898C9185FFEDCFCE017CDF40
:1015F000E8CFDF91CF91089580E090E0892B19F03A
:101600006ADF811125C080E090E0892B41F080E005
:1016100090E0892B21F00E94000081111CC080E025
:1016200090E0892B41F080E090E0892B21F00E942E
:101630000000811113C080E090E0892BA1F080E0D0
:1016400090E0892B81F00E94000081110AC008956A
:101650000E940000D8CF0E940000E1CF0E9400004D
:10166000EACF0C940000089590E0FC013197E2313C
:10167000F10508F04EC08827EE5AFE4F8F4F0C94AC
:101680005545809180008F7703C0809180008F7DC9
:1016900080938000089580918000877FF9CF84B582
:1016A0008F7702C084B58F7D84BD08958091B0008E
:1016B0008F7703C08091B0008F7D8093B000089534
:1016C000809190008F7707C0809190008F7D03C03C
:1016D00080919000877F8093900008958091A00072
:1016E0008F7707C08091A0008F7D03C08091A000FC
:1016F000877F8093A0000895809120018F7707C095
:10170000809120018F7D03C080912001877F80938D
:10171000200108953FB7F8948091760B9091770B54
:10172000A091780BB091790B26B5A89B05C02F3FEF
:1017300019F00196A11DB11D3FBFBA2FA92F982FF7
:101740008827820F911DA11DB11DBC01CD0142E072
:10175000660F771F881F991F4A95D1F708950F9339
:10176000FC019285908783858187A689B789119727
:1017700021F4621721F0401711F0628743878385B7
:101780008823D1F0828591110AC08823A9F080892D
:101790009189A289B3890197A109B10909C0811171
:1017A0000BC080899189A289B3890196A11DB11DC1
:1017B000808B918BA28BB38B0F910895EBE0F1E0BE
:1017C0008081877F80830895EBE0F1E080818860ED
:1017D000808308958E9808958E9A08951498089598
:1017E000149A089588980895889A08950E945747F2
:1017F0000F931F93CF93DF93EC018881998100971A
:1018000029F02A813B812617370788F48B016F5F07
:101810007F4F0E947346009761F0998388831B83F2
:101820000A832C813D81232B11F4FC01108281E07D
:1018300001C080E0DF91CF911F910F9108950F9328
:10184000CF93DF9380916C0B811173C081E0809303
:101850006C0B0E949016EC0106B126B1409100017C
:10186000609100010295017026FB222720F941704A
:101870006695617085589E4F72DF06B126B140B102
:1018800060B1017022FB222720F943FB442740F975
:1018900066956170CE018B569E4F61DF02B322B315
:1018A00040B160B1017022FB222720F9441F442778
:1018B000441F65FB662760F9CE0181559E4F4FDFBF
:1018C000FE01E259FF4F8081882361F0709780818B
:1018D0009181A281B3810196A11DB11D8083918365
:1018E000A283B383FE01E951FF4F8081882361F019
:1018F000709780819181A281B3810196A11DB11D54
:1019000080839183A283B383FE01E05AFE4F8081DE
:10191000882369F0C05BDE4F88819981AA81BB81F1
:101920000196A11DB11D88839983AA83BB83109260
:101930006C0BDF91CF910F910895EF92FF920F936F
:101940001F93CF93DF93FC012481358161157105CD
:1019500011F480E018C041155105A1F07B01EC01A4
:101960008A01020F131FB80143DF882391F32881F6
:1019700039818C819D81B701820F931F0E946D4731
:101980001D830C8381E0DF91CF911F910F91FF9018
:10199000EF900895EF92FF920F931F93CF93DF93F1
:1019A000CDB7DEB764970FB6F894DEBF0FBECDBFDC
:1019B0007C01CB01BA018E010F5F1F4F22E044E092
:1019C0000E947447BC01FC0101900020E9F73197A7
:1019D000AF01481B590BC701B0DF64960FB6F894EE
:1019E000DEBF0FBECDBFDF91CF911F910F91FF9052
:1019F000EF9008956115710549F0FB0101900020F9
:101A0000E9F73197AF01461B570B97CF80E0089558
:101A1000FB0144815581608171818FCFEF92FF92EC
:101A20000F931F93CF93DF93EC017B018A01BA01DF
:101A3000DFDE2881398181110DC02115310519F0B2
:101A4000C9010E942848198218821D821C821B82AB
:101A50001A8206C01D830C83B701C9010E946D471D
:101A6000CE01DF91CF911F910F91FF90EF900895DC
:101A7000FC01118210821382128215821482611578
:101A8000710549F0FB0101900020E9F73197AF01A2
:101A9000461B570BC3CF08951F920F920FB60F929C
:101AA00011240BB60F922F933F934F935F936F9335
:101AB0007F938F939F93AF93BF93EF93FF938AE8A6
:101AC0009BE012DDFF91EF91BF91AF919F918F91BC
:101AD0007F916F915F914F913F912F910F900BBE2E
:101AE0000F900FBE0F901F9018951F920F920FB678
:101AF0000F9211240BB60F922F938F939F93EF9316
:101B0000FF93E0919A0BF0919B0B8081E091A00BE9
:101B1000F091A10B82FD12C090818091A30B8F5F89
:101B20008F732091A40B821751F0E091A30BF0E08A
:101B3000E657F44F958F8093A30B01C08081FF91EE
:101B4000EF919F918F912F910F900BBE0F900FBE31
:101B50000F901F901895CF93DF93282F30E0F90155
:101B6000E451FD4F8491F901EA53FC4FD491F901FE
:101B7000E058FC4FC491CC2389F0811175DDEC2F26
:101B8000F0E0EE0FFF1FEA59FC4FA591B491EC91E4
:101B9000ED2381E090E021F480E002C080E090E05D
:101BA000DF91CF9108951F93CF93DF93282F30E0DB
:101BB000F901E451FD4F8491F901EA53FC4FD491AE
:101BC000F901E058FC4FC491CC23C1F0162F8111CC
:101BD0004BDDEC2FF0E0EE0FFF1FE45BFC4FA59117
:101BE000B4918FB7F894111105C09C91ED2FE09539
:101BF000E92302C0EC91ED2BEC938FBFDF91CF91E5
:101C00001F910895CF92DF92EF92FF920F931F934F
:101C1000CF93DF936C018B017A01EC01C359D44F50
:101C2000888187FF04C0FB011182108224C08CE0F0
:101C30008C9D90018D9D300D11248881A901480F44
:101C4000511D87FD5A958091BF0C90E048175907A8
:101C500094F48881A901480F511D87FD5A95CA0146
:101C6000FA01EE0FFF1F8E0F9F1FFC01E15DF34F86
:101C7000808186FD19C088818F5F88838CE08C9D70
:101C800090018D9D300D11248881A901480F511DAF
:101C900087FD5A958091BF0C90E048175907B4F41E
:101CA00088818C303CF112C08881280F311D87FD5E
:101CB0003A95F901EE0FFF1F2E0F3F1FF901E15D6D
:101CC000F34F808160E08F736EDFD5CFF8018081A4
:101CD0009181049680349C4918F480E49CE904C006
:101CE000F801808191810496F701918380838FEFC1
:101CF000888344C0F801408151818881B901680F0F
:101D0000711D87FD7A95CB01FB01EE0FFF1F8E0F32
:101D10009F1FFC01E15DF34F81819281840F951F2C
:101D2000F701918380838881A901480F511D87FDA8
:101D30005A95CA01FA01EE0FFF1F8E0F9F1FFC017B
:101D4000E15DF34F808186FF19C08881280F311D26
:101D500087FD3A95F901EE0FFF1F2E0F3F1FF90186
:101D6000E15DF34F808161E08F73DF91CF911F912F
:101D70000F91FF90EF90DF90CF9015CFDF91CF9133
:101D80001F910F91FF90EF90DF90CF90089560E04A
:101D9000FC01838508CF60E0FC01858104CF61E010
:101DA000FC01838500CF61E0FC018581FCCECF93EF
:101DB000DF9390E0FC01EA53FC4F2491FC01E058D2
:101DC000FC4F8491882361F190E0880F991FFC01FA
:101DD000EE5CFC4FC591D491FC01E45BFC4FA591F6
:101DE000B491611109C09FB7F8948881209582232E
:101DF0008883EC912E230BC0623061F49FB7F89476
:101E00003881822F809583238883EC912E2B2C930D
:101E10009FBF06C08FB7F894E8812E2B28838FBF11
:101E2000DF91CF9108958230910538F0880F991F86
:101E3000880F991F05970197F1F708958F929F9248
:101E4000AF92BF92CF92DF92EF92FF926B017C0133
:101E500061DC4B015C01C114D104E104F104E9F03F
:101E600059DCDC01CB0188199909AA09BB09883E14
:101E70009340A105B10578F321E0C21AD108E10829
:101E8000F10888EE880E83E0981EA11CB11CC114D5
:101E9000D104E104F10421F7DECFFF90EF90DF9051
:101EA000CF90BF90AF909F908F9008952FB7F894E8
:101EB0006091720B7091730B8091740B9091750B04
:101EC0002FBF08951F920F920FB60F9211242F93D8
:101ED0003F938F939F93AF93BF938091720B909199
:101EE000730BA091740BB091750B3091710B23E0C3
:101EF000230F2D3720F40196A11DB11D05C026E842
:101F0000230F0296A11DB11D2093710B8093720BBC
:101F10009093730BA093740BB093750B8091760B19
:101F20009091770BA091780BB091790B0196A11D40
:101F3000B11D8093760B9093770BA093780BB093A1
:101F4000790BBF91AF919F918F913F912F910F90FE
:101F50000FBE0F901F901895CF92DF92EF92FF92D5
:101F6000CF93DF93EC01603282E078070CF03DC044
:101F700077FD06C0653B71052CF064EB70E002C094
:101F800060E070E0898128E830E06901C81AD10872
:101F900087FDD394CC0CDD1CCC0CDD1C0D2C000C6F
:101FA000EE08FF088A8128E532E0281B310987FD09
:101FB0003395220F331F220F331FC901330FAA0B92
:101FC000BB0B9C01AD012C193D094E095F09DB01DA
:101FD0000E94924E24EB30E040E050E00E946C4EB4
:101FE000C20ED31EE41EF51EB6018881803380F533
:101FF000998148E850E0491B510997FD5395440FDA
:10200000551F440F551F6417750784F09A8128E502
:1020100032E0291B310997FD3395220F331F220F20
:10202000331FAB01261737070CF4A90142505109A1
:10203000440F551F2FB7F89490E0FC01EE0FFF1FDF
:102040008E0F9F1FFC01E15DF34F528341832FBF31
:10205000DF91CF91FF90EF90DF90CF9008951F9286
:102060000F920FB60F9211240BB60F922F933F933E
:102070004F935F936F937F938F939F93AF93BF9390
:10208000EF93FF9348E251E064E271E080E090E07A
:10209000B9DDFF91EF91BF91AF919F918F917F91AA
:1020A0006F915F914F913F912F910F900BBE0F90C9
:1020B0000FBE0F901F9018951F920F920FB60F92A0
:1020C00011240BB60F922F933F934F935F936F930F
:1020D0007F938F939F93AF93BF93EF93FF9348EAC0
:1020E00050E064EA70E083E090E08CDDFF91EF91D6
:1020F000BF91AF919F918F917F916F915F914F9120
:102100003F912F910F900BBE0F900FBE0F901F901D
:1021100018951F920F920FB60F9211240BB60F92C3
:102120002F933F934F935F936F937F938F939F93DF
:10213000AF93BF93EF93FF9348E950E064E970E0F9
:1021400082E090E05FDDFF91EF91BF91AF919F91B1
:102150008F917F916F915F914F913F912F910F9050
:102160000BBE0F900FBE0F901F9018951F920F92ED
:102170000FB60F9211240BB60F922F933F934F93EC
:102180005F936F937F938F939F93AF93BF93EF93DF
:10219000FF9348E850E064E870E081E090E032DDD1
:1021A000FF91EF91BF91AF919F918F917F916F912F
:1021B0005F914F913F912F910F900BBE0F900FBEEB
:1021C0000F901F9018951F920F920FB60F92112427
:1021D0000BB60F922F933F934F935F936F937F9321
:1021E0008F939F93AF93BF93EF93FF93E091240757
:1021F000F09125071995FF91EF91BF91AF919F91B4
:102200008F917F916F915F914F913F912F910F909F
:102210000BBE0F900FBE0F901F901895CF93DF93BA
:10222000EC01888198DC21E0892B09F420E02C87DF
:102230008C8191DC21E0892B09F420E02E878E89A6
:102240009F890197C1F48A8186DC21E0892B09F4FA
:1022500020E02D878E817FDC21E0892B09F420E0AE
:102260002F879C858D85981749F08E85821731F0D0
:102270009A878B8703C08C858A872B87DF91CF91C4
:102280000895CF93DF93FC01A489B589C08DD18DCA
:102290002089318942895389A03187E2B80759F0F2
:1022A0001A161B0644F40E94924E20E137E240E0E9
:1022B00050E00E946C4EDE010E94924EDF91CF9161
:1022C0000895FC011182108215821482108A118AED
:1022D000128A138A178A168A80E197E2958B848B7B
:1022E0001286108614861586168617860895CF9353
:1022F000DF93EC01FC01E859FF4F1082379781E032
:10230000808360E08D814FDC8F859889892B29F04F
:1023100060E08B85DF91CF9146CCDF91CF9108951E
:10232000CF93DF93EC018B8916DC892B11F08E891A
:1023300001C080E0DF91CF910895CF93DF93EC014E
:10234000898909DC892B11F08E8901C080E0DF9139
:10235000CF910895CF92DF92EF92FF920F931F9348
:10236000CF93DF937C016B018A01E9010E94D908B8
:10237000F601EE0FFF1FEE0FFF1FE85DF84F8081A3
:102380009181F701918380830E94D908000F111F6A
:10239000000F111FF801E85DF84F81E04081518185
:1023A00062817381413051056105710509F080E05A
:1023B000F70182870E94D908CC0FDD1FCC0FDD1FEB
:1023C000C85DD84F88819981AA81BB81F70182833A
:1023D0009383A483B5831682178210861186DF91BA
:1023E000CF911F910F91FF90EF90DF90CF900895C4
:1023F000CF92DF92EF92FF920F931F93CF93DF93D1
:10240000EC0186E390E09E8B8D8B87E390E0988FC4
:102410008F8B86E290E09A8F898F8AE190E09C8F83
:102420008B8F8CE190E09E8F8D8F88E190E098A358
:102430008F8F83E090E09AA389A382E090E09CA331
:102440008BA3FE01E757FF4F8CE390E096838583D3
:102450008DE390E09087878388E390E0928781877F
:102460001486138616861586108A17868EE090E0ED
:10247000928B818B8FE090E0948B838BE758FF4F9A
:102480008EE290E09683858380E390E09087878357
:102490008EE390E0928781871486138616861586D0
:1024A000108A178682E190E0928B818B83E190E025
:1024B000948B838BE852FF4F1182108232961182E7
:1024C0001082329611821082CE010E949925CE018F
:1024D0000E94B4326E0185E8C81A8EEFD80A80E1F6
:1024E00090E0F6019183808381E190E0958384837D
:1024F0008FE190E09383828381E290E097838683EB
:10250000C6018CDEF60182858087838581877E0106
:10251000FBE6EF1AFEEFFF0A87E190E0F7019183F7
:10252000808389E190E09583848383E290E09383C4
:10253000828385E290E097838683C7016FDEF7018F
:1025400082858087838581878E0101551E4F8BE1AF
:1025500090E0F801918380838DE190E095838483FE
:1025600087E290E09383828389E290E09783868379
:10257000C80154DEF8018285808783858187E35016
:10258000FF4F808191813C97208131813697408136
:102590005181F601578B468B358B248B019719F4AB
:1025A0008FEF9FEF03C081E090E0F601918F808F65
:1025B000FE01E255FD4F808191813C972081318160
:1025C000369740815181F701578B468B358B248B91
:1025D000019719F48FEF9FEF03C081E090E0F701BE
:1025E000918F808FFE01E055FD4F808191813C9756
:1025F00020813181C256DD4F48815981F801578BC6
:10260000468B358B248B019719F48FEF9FEF03C016
:1026100081E090E0F801918F808FDF91CF911F9141
:102620000F91FF90EF90DF90CF9008952F923F92FF
:102630004F925F926F927F928F929F92AF92BF92D2
:10264000CF92DF92EF92FF920F931F93CF93DF937E
:10265000CDB7DEB7C957D1090FB6F894DEBF0FBEAC
:10266000CDBF8C01FC011082118212821382148270
:10267000158216821782108611861286138614869A
:102680001586168617862C01F0E14F0E511CC201EB
:102690000E941D32680189E8C80ED11CC6010E9443
:1026A0001D327801EEEFEE1AFE0AC7010E941D32BC
:1026B0003801F5E86F1AFEEF7F0AC30102DE480118
:1026C0008BE6881A8EEF980AC401FBDD5801E1E51C
:1026D000AE1AEEEFBE0AC501F4DD68EC73E0C80186
:1026E00087539E4FC5D9F801E153FE4F11821082E6
:1026F00032961182108232961182108232961182A5
:102700001082329610823196108231961082319664
:1027100011821082329611821082329611821082BA
:102720003296108231961082319610823196108244
:1027300011821282138234961082118212821382C5
:102740003496108211821282138234961082118282
:10275000128213823496108211821282138234966E
:102760001082118212821382349610821182128298
:102770001382349610821182128213823496108250
:102780001182128213823496108211821282138275
:102790003496108211821282138234961082118232
:1027A000128213823496108211821282138234961E
:1027B0001082118212821382349610821182128248
:1027C000138234961082319610823196108231969F
:1027D0001082118212821382349610821182128228
:1027E00013823496108211821282138234961082E0
:1027F0003196108231961082319610823196108275
:102800003196108231961082319610823196108264
:102810003196108231961082319610823196108254
:102820003196108231961082319610823196108244
:102830003196108231961082319610823196108234
:102840003196108211821282138234961082118284
:102850001282138234961082118212821382D8015E
:10286000A15BBD4F8CE0EAE1F3E001900D928A9507
:10287000E1F7F801E55AFD4F1082118212821382AE
:102880003496108211821282138234961082118241
:102890001282138234961182108232961182108233
:1028A0003296118210823296108211821282138225
:1028B0003496108211821282138234961082118211
:1028C00012821382349610821182128213823496FD
:1028D0001082118212821382349610821182128227
:1028E00013823496118210823296118210823296AF
:1028F00011821082329610821182128213823496D3
:1029000010821182128213823496108211821282F6
:10291000138234961082319610823196108231964D
:1029200011821082329611821082329611821082A8
:102930003296118210823296118210823296118262
:102940001082329611821082329611821082329653
:102950001182108232961182108232961182108278
:102960003296118210823296118210823296118232
:1029700010821801FAE42F1AFDEF3F0AF1011082CC
:10298000CE0101960E941D3289E7FE013196D201E7
:1029900001900D928A95E1F7CE0101960E941D32B9
:1029A00089E7FE013196D60101900D928A95E1F7F3
:1029B000CE0101960E941D3289E7FE013196D701B2
:1029C00001900D928A95E1F788E5F801808B89E501
:1029D000F60180838AE5F7018083CE01019671DCE0
:1029E0008AE1FE013196D30101900D928A95E1F7BB
:1029F000CE01019666DC8AE1FE013196D401019098
:102A00000D928A95E1F7CE0101965BDC8AE1FE0129
:102A10003196D50101900D928A95E1F7C801E8DC65
:102A2000F1011082C758DF4F0FB6F894DEBF0FBE1A
:102A3000CDBFDF91CF911F910F91FF90EF90DF906D
:102A4000CF90BF90AF909F908F907F906F905F904E
:102A50004F903F902F9008950F931F93CF93DF9344
:102A60008B01EA0182E393E00E94A83982E894E0B6
:102A70000E94A839F80180810E94E939CE010E94A4
:102A8000EA3A0E94EB24DF91CF911F910F910C94B1
:102A9000F523CF92DF92EF92FF920F931F93CF9384
:102AA000DF93CDB7DEB728970FB6F894DEBF0FBE21
:102AB000CDBF8B016A0187539E4F7C016EE273E0AC
:102AC0000E94FA0C62E874E0C7010E94FA0CF80157
:102AD000808189831A8241E050E08E010F5F1F4F91
:102AE000B801C7010E949D0C4AE0B801C6010E94CE
:102AF000ED48F80101900020E9F73197AF01401B44
:102B0000510BB801C7010E949D0C0E94EB24BC012F
:102B1000C8010E94AF23B801C7010E94080D898136
:102B20009A810E94284828960FB6F894DEBF0FBEFF
:102B3000CDBFDF91CF911F910F91FF90EF90DF906C
:102B4000CF900895FC01DB01AE59BF4F8C918823D3
:102B500019F022E030E002C020E030E0DB01AC59A7
:102B6000BF4F8C91882311F023E030E0DB01AD5999
:102B7000BF4F8C91882311F024E030E0DB01AB598A
:102B8000BF4F8C91882311F026E030E0DA018D915F
:102B90009C918217930721F091E0121613060CF016
:102BA00090E0DA012D933C93992319F0A901CF010C
:102BB00070CF08958F929F92AF92BF92CF92DF9283
:102BC000EF92FF920F931F93CF93DF93EC018AE272
:102BD00093E00E94A83981E994E00E94A8396E012F
:102BE00085E8C81A8EEFD80AC6014BDB0E94404D1B
:102BF0004B015C01FE01E15BFD4F608171818281CF
:102C000093810E94404D9B01AC01C501B4010E941B
:102C1000C94542E00E941B3A81EA94E00E94A8392B
:102C20007E01EBE6EE1AEEEFFE0AC7012ADB0E94F8
:102C3000404D4B015C01FE01ED5AFD4F60817181F9
:102C4000828193810E94404D9B01AC01C501B4017A
:102C50000E94C94542E00E941B3A81EB94E00E9429
:102C6000A8398E0101551E4FC8010BDB0E94404D53
:102C70004B015C01C95ADD4F688179818A819B8152
:102C80000E94404D9B01AC01C501B4010E94C945A1
:102C900042E00E941B3A0E94EB240E94F52386E248
:102CA00093E00E94A83981E994E00E94A839F601D6
:102CB000A08DB18D20893189428953890E94924E1D
:102CC0000E94F43981EA94E00E94A839F701A08DAE
:102CD000B18D20893189428953890E94924E0E9488
:102CE000F43981EB94E00E94A839F801A08DB18DF0
:102CF00020893189428953890E94924E0E94F43979
:102D00000E94EB24DF91CF911F910F91FF90EF90E4
:102D1000DF90CF90BF90AF909F908F900C94F52351
:102D2000CF93DF9380917E0B90917F0B892B51F491
:102D300087EB92E00E949347EC0178DCD0937F0B05
:102D4000C0937E0B80917E0B90917F0BDF91CF9192
:102D50000895CF93DF93EC012AEC30E04BEC50E088
:102D600069EC70E0F7DA2EEC30E04FEC50E06DECFF
:102D700070E0CE010C96EEDA24ED30E045ED50E047
:102D800063ED70E0CE014896E5DA28ED30E049EDDC
:102D900050E067ED70E0CE018496DCDA2EED30E095
:102DA0004FED50E06DED70E0CE01C096DF91CF9118
:102DB000D1CACF93DF9380917C0B90917D0B892BAF
:102DC000E9F48CE390E00E949347EC01FC01CC967F
:102DD000118210823C96E817F907D1F71982188200
:102DE0001D861C86198E188E1DA21CA219AA18AA4F
:102DF000CE01AFDFD0937D0BC0937C0B80917C0B19
:102E000090917D0BDF91CF910895EF92FF920F93F8
:102E10001F93CF93DF93162F072F7A01411551058A
:102E200059F4862F0E94AB0D31E020E0019709F0A4
:102E300030E0C32FD22F26C04130510509F5262F8F
:102E4000663310F02AEC260F80917B00922F987049
:102E5000877F892B80937B002770206420937C00E0
:102E600080917A00806480937A0080917A0086FD58
:102E7000FCCFC091780080917900D0E0D82B02C0BF
:102E8000C0E0D0E082E0E816F10410F585EE94E0B1
:102E90000E94A83982E894E00E94A8398FEB94E060
:102EA0000E94A839812F902F0E94EA3A82E894E08C
:102EB0000E94A83981EC94E00E94A839CE010E94BA
:102EC000EA3A0E94EB240E94F52380E090E002C0E1
:102ED00081E090E0DF91CF911F910F91FF90EF90F3
:102EE00008950F931F93CF93DF938B01EA01AB01FA
:102EF000415051094433510508F0D4C02230310506
:102F000008F0D0C048E3429FF001439FF00D112428
:102F1000E60FF71FE80FF91F81E08083232B11F4E0
:102F20006C2F07C061E0802F0E94D70E209739F4E4
:102F300060E0802F0E94D30D80E090E0B5C0CF3FCD
:102F4000D10509F4ADC0F801E451FD4FE4918E2F95
:102F500090E0FC013197E231F10508F09DC088272F
:102F6000EC59FE4F8F4F0C94554584B5806884BD55
:102F7000C7BDE2CF84B5806284BDC8BDDDCF80917E
:102F80008000806880938000D0938900C09388007F
:102F9000D3CF80918000806280938000D0938B009B
:102FA000C0938A00C9CF80918000886080938000A0
:102FB000D0938D00C0938C00BFCF8091B00080680B
:102FC0008093B000C093B300B7CF8091B00080620F
:102FD0008093B000C093B400AFCF80919000806820
:102FE00080939000D0939900C0939800A5CF8091D2
:102FF0009000806280939000D0939B00C0939A00D1
:103000009BCF80919000886080939000D0939D002A
:10301000C0939C0091CF8091A00080688093A00015
:103020008091A0008F7B8093A000D093A900C093D3
:10303000A80082CF8091A00080628093A000D093EE
:10304000AB00C093AA0078CF8091A00088608093E5
:10305000A000D093AD00C093AC006ECF8091200152
:10306000806880932001D0932901C093280164CF08
:1030700080912001806280932001D0932B01C09326
:103080002A015ACF80912001886080932001D0933B
:103090002D01C0932C0150CFC038D1050CF448CF7E
:1030A00061E047CF81E090E0DF91CF911F910F91D8
:1030B000089580917A0B90917B0B892BA1F480E786
:1030C00090E00E949347FC01F9969C0123593F4FE1
:1030D000DF01D8971C921192E217F307C9F790937A
:1030E0007B0B80937A0B80917A0B90917B0B0895E8
:1030F0000F931F93CF93DF93FC0120813181211522
:103100003105D1F1EC01822F0E94AB0D21E0892B1A
:1031100009F420E02B876A85261729F01E821F827A
:10312000188619860BC08E819F81A885B985019666
:10313000A11DB11D8E839F83A887B9870E811F8132
:10314000288539858A819B81AC81BD810817190743
:103150002A073B078CF081E0682788810E94D30D05
:103160000990D881C02DA5DF40E050E0BE01DF917D
:10317000CF911F910F9149CEDF91CF911F910F9168
:103180000895683671050CF050C0653671050CF075
:103190008CC06C32710554F5693271050CF085C034
:1031A0006831710594F46F3071050CF07EC06630A3
:1031B000710544F4623071050CF077C0672B09F09B
:1031C00072C073C06B5071096BC0623271053CF400
:1031D0006F3171050CF069C06951710961C06452A9
:1031E00071096230710508F05EC05FC06A33710515
:1031F0007CF4673371050CF058C06D3271050CF426
:1032000052C0603371050CF450C06353710948C05B
:10321000643471053CF4613471050CF046C06D53A3
:1032200071093EC0675471093BC060397105F4F4FF
:103230006D387105D4F56637710564F4633771052F
:10324000A4F5693671057CF16C36710574F16F5621
:10325000710926C06038710534F46D3771052CF59D
:10326000695771091DC0635871091AC0603D710525
:1032700064F46D3C7105CCF461397105A4F06439D6
:1032800071059CF0695C71090BC06A3D710534F4ED
:10329000673D710554F4635D710902C06D5D71098C
:1032A0006330710510F080E0089581E008952F9259
:1032B0003F924F925F926F927F928F929F92AF92C6
:1032C000BF92CF92DF92EF92FF920F931F93CF9313
:1032D000DF93CDB7DEB7E4970FB6F894DEBF0FBE2D
:1032E000CDBF1C012A013B0109871A872B873C8728
:1032F0002C960EAD1FAD2C97FC01E15BFD4F60815C
:103300007181828193810E94404D9B01AC01C30178
:10331000B2010E949F4D0E9439466B8B7C8B8D8B36
:103320009E8BF101ED5AFD4F608171818281938105
:103330000E94404D9B01AC0169857A858B859C85F7
:103340000E949F4D0E9439466F8B788F898F9A8F8C
:10335000F101E95AFD4F60817181828193810E9460
:10336000404D9B01AC01C701B6010E949F4D0E94D8
:1033700039466B8F7C8F8D8F9E8F0E94560F6D8785
:103380007E878F87988BF101ED52FE4F118210825C
:103390003296118210823E96A114B10461F0C501EB
:1033A000A0E0B0E04081518162817381841795076C
:1033B000A607B70714F0A080B180F101E951FE4FD4
:1033C0008114910461F0C401A0E0B0E0408151811A
:1033D0006281738184179507A607B70714F0808070
:1033E0009180F101E551FE4F0115110561F0C80111
:1033F000A0E0B0E04081518162817381841795071C
:10340000A607B70714F0008111819101205F3F4F9B
:103410003A8B298BC501A0E0B0E0F10187A390A70A
:10342000A1A7B2A72101F9E84F0E511CA12CB12C84
:10343000D20157968D929D92AD92BC925A973101CE
:10344000BEEF6B1A7B0A20E030E0F301078B108F90
:10345000218F328F0E94EB240E94EB240E94EB24E8
:103460000E94EB244091B00A5091B10A6091B20AD7
:103470007091B30A49AB5AAB6BAB7CAB0E94EB24A7
:103480008091B40A9091B50AA091B60AB091B70A9A
:1034900089879A87AB87BC870E94EB248090B80A03
:1034A0009090B90AA090BA0AB090BB0AF101E55A0F
:1034B000FD4F108211821282138234961082118283
:1034C00012821382349610821182128213823496F1
:1034D00011821082329611821082329611821082ED
:1034E000329649A95AA96BA97CA94083518362836A
:1034F0007383349689859A85AB85BC858083918357
:10350000A283B383349680829182A282B3822D9665
:10351000EFAC2D970B891C892D893E8989899A8961
:103520000E94B32D2E96EFAC2E970F89188D298D02
:103530003A8D49855A856B857C85C2010E94B32DE1
:103540002F96EFAC2F970B8D1C8D2D8D3E8DB501D9
:10355000A401C3010E94B32DD10151961C92F10127
:10356000E657FF4F1082E758FF4F1082C1010E94BB
:103570008132C1010E94853289899A890E94FB317A
:10358000C2010E94FB31C3010E94FB31F101E652EE
:10359000FE4FFAA3E9A381E090E09183808371015B
:1035A000F4E2EF1AFEEFFF0AD7018D939C9381019D
:1035B00002521E4FF8019183808341E050E06989F7
:1035C0007A89C10166DAD7014D915C91B201C101DE
:1035D00060DAF80140815181B301C1015ADA11E08A
:1035E000F101EA54FD4F108389899A890E949E2D2A
:1035F000C2010E949E2DC3010E949E2D64E670E0D0
:1036000080E090E00E941E0FC10189529E4FDC01B4
:103610001C9311961C93A10147525E4FFA0110832F
:103620002D96FFAD2D97F1110FC02E962FAD2E9731
:10363000211105C02F963FAD2F97332339F191010A
:1036400022593F4FF90110822E96FFAD2E97F111AE
:1036500005C0910129513F4FF90110822F96FFAD0E
:103660002F97F11105C09101205A3E4FF9011082A8
:103670002D962FAD2D97FC0120832E963FAD2E97D2
:103680003C932F96EFAD2F97DA01EC9389899A89B5
:103690000E945F2FC2010E945F2FC3010E945F2F13
:1036A00089899A890E94B42EC2010E94B42EC30156
:1036B0000E94B42E0E94EB24DC011C968C918B8B13
:1036C0001A861986F101E952FE4FF88FEF8B9101AE
:1036D00028523E4F3C8F2B8FA10147525E4F58A37B
:1036E0004F8FC10186529E4F9AA789A7D101A4523C
:1036F000BE4FBCA7ABA73796FEA7EDA72756314014
:1037000038A72FA342545F4F58AB4FA78451914025
:103710009CA38BA3AD59B109BEA3ADA3EF89F88DCE
:10372000808181110BC0AB8DBC8D8C91811106C045
:10373000EF8DF8A18081882309F45DC3FB89F11125
:103740005AC349A55AA569897A89C101FBD94BA5F4
:103750005CA5B201C101F6D94DA55EA5B301C101B9
:10376000F1D989899A890E941E2FC2010E941E2FB9
:10377000C3010E941E2FEFA1F8A58081882331F19B
:1037800089899A890E945F2F8FA498A85101F5E733
:10379000AF1AFDEFBF0A61012AE5C21A2DEFD20A66
:1037A000710137E8E31A3DEFF30A810103591D4F18
:1037B0009101255A3D4FA10145585E4F69897A898B
:1037C000C1010E94962CAFA1B8A51C92F101E6514F
:1037D000FF4FF887EF838081882339F1C2010E946F
:1037E0005F2F4101F8E68F1AFDEF9F0A510121E793
:1037F000A21A2DEFB20A610138E5C31A3DEFD30AD0
:10380000710143E8E41A4DEFF40A81010F581D4F8E
:103810009101215A3D4FA1014B565E4FB201C101AA
:103820000E94962CAF81B8851C92F101ED59FE4F94
:10383000F887EF838081882339F1C3010E945F2FCD
:103840004101F7E68F1AFDEF9F0A51012DE6A21AFA
:103850002DEFB20A610136E5C31A3DEFD30A7101BB
:103860004FE7E41A4DEFF40A81010B581D4F910107
:103870002D593D4FA10141555E4FB301C1010E9439
:10388000962CAF81B8851C92810102591F4FF80117
:103890008081882309F43EC0E95EFD4F608171811B
:1038A000072E000C880B990B0E94404D9B01AC0128
:1038B000F101E55AFD4F60817181828193810E94FF
:1038C0006B4618163CF5D8011C926EE474E0810139
:1038D00007531E4FC8010E94FA0C67E275E0C80149
:1038E0000E94FA0C66EC73E0C8010E94FA0C2D9657
:1038F000BFAD2D97BB2309F471C3F101E558FE4F0D
:10390000108A118A128A138AEE52F14010821182B3
:1039100012821382810109511F4FD8018C91882393
:1039200009F43FC0F101E957FD4F60817181072E15
:10393000000C880B990B0E94404D9B01AC01F101DA
:10394000E15AFD4F60817181828193810E946B46B3
:1039500018163CF5D8011C926EE474E081010753FF
:103960001E4FC8010E94FA0C6FE475E0C8010E9466
:10397000FA0C66EC73E0C8010E94FA0C2E96BFADFB
:103980002E97BB2309F42FC3F101EB56FE4F108A8B
:10399000118A128A138AEBA1FCA110821182128271
:1039A00013828101005A1E4FD8018C91882309F49B
:1039B0003FC0F101E757FD4F60817181072E000C78
:1039C000880B990B0E94404D9B01AC01F101ED5910
:1039D000FD4F60817181828193810E946B46181630
:1039E0003CF5D8011C926EE474E0810107531E4F30
:1039F000C8010E94FA0C67E775E0C8010E94FA0C42
:103A000066EC73E0C8010E94FA0C2F96BFAD2F97A9
:103A1000BB2309F4EDC2F101E155FE4F108A118A72
:103A2000128A138AEDA1FEA11082118212821382E2
:103A300060E089899A890E94292E882369F0F10122
:103A4000E35BFF4F1082118212821382E25DFE4F10
:103A5000108A118A128A138A60E0C2010E94292EFC
:103A6000882371F0ABA1BCA11D921D921D921C92E6
:103A70001397F101EB56FE4F108A118A128A138AAE
:103A800060E0C3010E94292E882369F0EDA1FEA108
:103A90001082118212821382F101E155FE4F108AC9
:103AA000118A128A138AF101E259FF4F8081AF898E
:103AB000B88D8C93E758FF4F8081EB8DFC8D808310
:103AC000F101E05AFE4F8081AF8DB8A18C93E35194
:103AD000F1404081518162817381EBA1FCA1808022
:103AE0009180A280B380ADA1BEA1CD90DD90ED907C
:103AF000FC9049AB5AAB6BAB7CAB6DD749A95AA9CB
:103B00006BA97CA94093B00A5093B10A6093B20AA2
:103B10007093B30A60D78092B40A9092B50AA092CB
:103B2000B60AB092B70A57D7C092B80AD092B90A6B
:103B3000E092BA0AF092BB0AC1010E948132EF8979
:103B4000F88D8081882309F44AC00E94560F2D8584
:103B50003E854F855889621773078407950760F47F
:103B60000E94560F2D853E854F8558896217730731
:103B700084079507A0F51EC00E94560F6B017C01BB
:103B80002D853E854F855889C21AD30AE40AF50A65
:103B9000F101ED5BFD4F2081318142815381A8EE1F
:103BA000B3E00E94884E6C157D058E059F0508F4D4
:103BB00024C2D6CF0E94560F6B017C01F101ED5B50
:103BC000FD4F2081318142815381A8EEB3E00E94F4
:103BD000884E6C157D058E059F0508F40EC2AB8DD1
:103BE000BC8D8C91882309F44AC00E94560F2D8504
:103BF0003E854F855889621773078407950760F4DF
:103C00000E94560F2D853E854F8558896217730790
:103C100084079507A0F51EC00E94560F6B017C011A
:103C20002D853E854F855889C21AD30AE40AF50AC4
:103C3000F101ED5BFD4F2081318142815381A8EE7E
:103C4000B3E00E94884E6C157D058E059F0508F433
:103C5000E0C1D6CF0E94560F6B017C01F101ED5BF4
:103C6000FD4F2081318142815381A8EEB3E00E9453
:103C7000884E6C157D058E059F0508F4CAC1AF8D71
:103C8000B8A18C91882309F44AC00E94560F2D8553
:103C90003E854F855889621773078407950760F43E
:103CA0000E94560F2D853E854F85588962177307F0
:103CB00084079507A0F51EC00E94560F6B017C017A
:103CC0002D853E854F855889C21AD30AE40AF50A24
:103CD000F101ED5BFD4F2081318142815381A8EEDE
:103CE000B3E00E94884E6C157D058E059F0508F493
:103CF0009CC1D6CF0E94560F6B017C01F101ED5B98
:103D0000FD4F2081318142815381A8EEB3E00E94B2
:103D1000884E6C157D058E059F0508F486C18AE8DE
:103D20009BE00E945F0A181619065CF58AE89BE082
:103D30000E943D0A8F7D8534910519F569EE74E086
:103D4000C10187539E4F0E94FA0C82E493E00E94C7
:103D5000A83941D64AD5F101E259FF4F1082E75800
:103D6000FF4F1082E758FF4F1082AF89B88D1C9229
:103D7000EB8DFC8D1082AF8DB8A11C92B1E0BB8B96
:103D800004C0E985FA853197A9F46EEF74E0C101AA
:103D900087539E4F0E94FA0CAF89B88D1C92EB8D11
:103DA000FC8D1082AF8DB8A11C92E1E0F0E0FA87A3
:103DB000E98702C01A861986C1010E945E39F101A5
:103DC000EB52FE4F808191810196918380838D32E9
:103DD00091400CF4A3CCD101A353BE4F8D919C9183
:103DE0001197892B09F09ACC14968D919C91892B6F
:103DF00009F427C193CC810103531E4FD8018D9143
:103E00009C91892B21F0C1010E945E39F7CF8EE091
:103E100095E00E94A8392D96BFAD2D97BB23F1F0F8
:103E2000E985FA85EF2BD1F4FB89F1113CC08EE3D3
:103E300093E00E94A839CFD5D8D42E962FAD2E97D7
:103E4000222361F18AE393E00E94A839C4D5CDD43E
:103E50002F963FAD2F9731111AC025C02E964FAD2A
:103E60002E97442341F089859A85892B21F49B89DB
:103E7000911119C0E7CF2F96AFAD2F97AA2399F0D4
:103E8000E985FA85EF2B79F4FB89F1110CC086E303
:103E900093E00E94A8399FD5A8D405C02F969FAD66
:103EA0002F979111F4CF85E090E0A9A1BAA18D934D
:103EB0009C93910124523E4F3E872D87D9018D93CB
:103EC0009C93810102521E4FF8019183808345E04B
:103ED00050E069897A89C1010E944915AD85BE8586
:103EE0004D915C91B201C1010E944915F8014081D8
:103EF0005181B301C1010E944915C1010E9489325B
:103F0000F101E35BFF4F4081518162817381E7588A
:103F1000FF4FC080D180E280F380E758FF4F808060
:103F20009180A280B38049AB5AAB6BAB7CAB53D5CD
:103F300049A95AA96BA97CA94093B00A5093B10A28
:103F40006093B20A7093B30A46D5C092B40AD09275
:103F5000B50AE092B60AF092B70A3DD58092B80A47
:103F60009092B90AA092BA0AB092BB0AC1010E940B
:103F70008132C1010E9485322ED58AD4C1010E94AE
:103F8000DA15A9A1BAA11D921C92ED85FE851182B8
:103F90001082D8011D921C9240E050E069897A8914
:103FA000C1010E944915ED85FE8540815181B20114
:103FB000C1010E944915D8014D915C91B301C10125
:103FC0000E944915C1010E948932BB89BB2309F4B3
:103FD00032C101D521E0FC0124872DC1E1E0F0E0F0
:103FE000FA87E98797CCE1E0F0E0FA87E987D9CC56
:103FF000E1E0F0E0FA87E9871BCD6FE975E0C101E8
:1040000087539E4F0E94FA0C21E030E03A872987BF
:10401000E6CD64EB75E0C10187539E4F0E94FA0C18
:1040200041E050E05A8749872ACE69EC75E0C1012A
:1040300087539E4F0E94FA0C81E090E09A8789870F
:104040006ECE11821082F101ED52FE4F808191817E
:10405000009749F466E473E0810107531E4FC801DD
:104060000E94FA0CC5C0019709F0D1C0B4D48C01EC
:10407000FC0180819181A281B381181619061A066C
:104080001B0644F081E090E0A0E0B0E080839183E3
:10409000A283B383F80184819581A681B781181624
:1040A00019061A061B0644F081E090E0A0E0B0E09B
:1040B00084839583A683B783F80180859185A28543
:1040C000B385181619061A061B0644F081E090E025
:1040D000A0E0B0E080879187A287B38768EC73E0A7
:1040E000CE0101960E94380D6AE075E0CE0101967E
:1040F0000E94FA0C61E974E0CE0101960E94FA0C6C
:104100006091B00A7091B10A8091B20A9091B30A9D
:104110000E94404D6B017C01D8016D917D918D9184
:104120009C910E94404D9B01AC01C701B6010E94C9
:10413000C945AB01BC01CE0101960E94CA0C61EADF
:1041400074E0CE0101960E94FA0C6091B40A70915D
:10415000B50A8091B60A9091B70A0E94404D6B0152
:104160007C01F80164817581868197810E94404DB0
:104170009B01AC01C701B6010E94C945AB01BC015E
:10418000CE0101960E94CA0C61EB74E0CE0101964B
:104190000E94FA0C6091B80A7091B90A8091BA0A2B
:1041A0009091BB0A0E94404D6B017C01D80118968A
:1041B0006D917D918D919C911B970E94404D9B012B
:1041C000AC01C701B6010E94C945AB01BC01CE01DB
:1041D00001960E94CA0CBE016F5F7F4F8101075399
:1041E0001E4FC8010E94080D89819A810E942848AB
:1041F000F2D3BC01CE010196B2D2BE016F5F7F4FF8
:10420000C8010E94080D89819A810E942848F10105
:10421000ED52FE4F808191810196823091051CF410
:104220009183808302C011821082F101EF52FE4F10
:104230001182108273CA8CE195E00E94A8398985A9
:104240009A850E94EA3A86EC93E00E94A839C3D38B
:1042500029853A853093270720932607C901E496DC
:104260000FB6F894DEBF0FBECDBFDF91CF911F9187
:104270000F91FF90EF90DF90CF90BF90AF909F9005
:104280008F907F906F905F904F903F902F90089508
:10429000EF92FF920F931F93CF93DF93FB01E2A85E
:1042A000F3A802A113A1C68DD78D0E9459189701BA
:1042B000A801BE010E94711780E090E0DF91CF91CC
:1042C0001F910F91FF90EF9008956F927F928F92C0
:1042D0009F92AF92BF92CF92DF92EF92FF920F9395
:1042E0001F93CF93DF93FB01E2A8F3A886A497A4C2
:1042F000A0A8B1A8C6A0D7A062A073A0068D178DF4
:104300000E945918EC019701A301B8010E9471178E
:10431000C501B4010E941E0F9701A601B801CE018C
:104320000E94711780E090E0DF91CF911F910F9173
:10433000FF90EF90DF90CF90BF90AF909F908F90C5
:104340007F906F9008950C9428480C9428480C9402
:1043500028480C9428480C9428480C9428480C941D
:1043600028480C9428480C9428480C9428480C940D
:1043700028480C9428480C9428481F93CF93DF9327
:104380001F92CDB7DEB7FB0162A9168D69830E942B
:1043900059186981812F0E94D70E80E090E00F901C
:1043A000DF91CF911F9108950F931F93CF93DF93C8
:1043B000FB0102A913A9C68DD78D0E945918A80127
:1043C000BE010E94051780E090E0DF91CF911F9120
:1043D0000F910895662319F087ED93E002C080EDF8
:1043E00093E00C94A839CF93DF93FB01C68DD78D52
:1043F0000E94D908BE010E94960880E090E0DF91FB
:10440000CF910895EF92FF920F931F93CF93DF9375
:1044100000D01F92CDB7DEB7FB0122A133A144A18A
:1044200055A1068D178D29833A834B835C830E94A7
:10443000D9087C01FC018281938129813A814B81D9
:104440005C818F30F7E29F072CF40196F70193838C
:10445000828303C0F70113821282B801C701298346
:104460003A834B835C830E94C11829813A814B8136
:104470005C818823A1F0F801EE0FFF1FEE0FFF1FF4
:10448000E85DF84F2083318342835383B801C7012D
:104490000E944708B801C7010E94960804C083EC37
:1044A00094E00E94A8390E94D9160E94A91680E0C3
:1044B00090E00F900F900F900F90DF91CF911F9190
:1044C0000F91FF90EF9008958F929F92AF92BF92BD
:1044D000CF92DF92EF92FF920F931F930E9490165C
:1044E00062E070E00E948F34892BD1F40E94901614
:1044F00021E02F931F921F921F921F92812C912CCB
:10450000A12CB12CC12CD12C760197018601B701C9
:10451000A6010E9457190F900F900F900F900F90C7
:1045200080E090E01F910F91FF90EF90DF90CF908F
:10453000BF90AF909F908F9008958F929F92AF926F
:10454000BF92CF92DF92EF92FF920F931F930E9440
:10455000901661E070E00E948F34892BD1F40E94A4
:1045600090161F9221E02F931F921F921F92812C71
:10457000912CA12CB12CC12CD12C76019701860154
:10458000B701A6010E9457190F900F900F900F903E
:104590000F9080E090E01F910F91FF90EF90DF90DF
:1045A000CF90BF90AF909F908F9008958F929F92E1
:1045B000AF92BF92CF92DF92EF92FF920F931F9331
:1045C0000E94901660E070E00E948F34892BD1F435
:1045D0000E9490161F921F9221E02F931F921F920C
:1045E000812C912CA12CB12CC12CD12C76019701BE
:1045F0008601B701A6010E9457190F900F900F90E6
:104600000F900F9080E090E01F910F91FF90EF903E
:10461000DF90CF90BF90AF909F908F9008958F9232
:104620009F92AF92BF92CF92DF92EF92FF920F9341
:104630001F930E94901621E02F931F921F921F92AA
:104640001F92812C912CA12CB12CC12CD12C760144
:1046500097018601B701A6010E9457190F900F908C
:104660000F900F900F9080E090E01F910F91FF90BE
:10467000EF90DF90CF90BF90AF909F908F90089574
:104680008F929F92AF92BF92CF92DF92EF92FF9262
:104690000F931F930E9490161F9221E02F931F9259
:1046A0001F921F92812C912CA12CB12CC12CD12CAA
:1046B000760197018601B701A6010E9457190F9054
:1046C0000F900F900F900F9080E090E01F910F914E
:1046D000FF90EF90DF90CF90BF90AF909F908F9022
:1046E00008958F929F92AF92BF92CF92DF92EF92F6
:1046F000FF920F931F930E9490161F921F9221E02A
:104700002F931F921F92812C912CA12CB12CC12C84
:10471000D12C760197018601B701A6010E94571995
:104720000F900F900F900F900F9080E090E01F91EE
:104730000F91FF90EF90DF90CF90BF90AF909F9040
:104740008F900895089508950895089508950895FF
:104750000895089508950895089508950895EF928D
:10476000FF920F931F93CF93DF93CDB7DEB72E97B2
:104770000FB6F894DEBF0FBECDBF8C0168EC73E0BE
:104780000E94380D6EED75E0C8010E94FA0C609130
:10479000AC0A7091AD0A8091AE0A9091AF0A2AE0FE
:1047A000AE014F5F5F4F7A010E94F748F701019019
:1047B0000020E9F73197AF014E195F09B701C80131
:1047C0000E949D0C66EC73E0C8010E94FA0CC801BF
:1047D0002E960FB6F894DEBF0FBECDBFDF91CF91FE
:1047E0001F910F91FF90EF9008958EED95E00E943C
:1047F000A8396091AC0A7091AD0A8091AE0A90918F
:10480000AF0A0E94F43986EC93E00C94A8390F9318
:104810001F93CF93DF93EC0181EE95E00E94A839BE
:1048200085EE95E00E94A83904E81BE0F80160815C
:10483000CE01D0DD89EE95E00E94A839F8016181B2
:10484000CE01C8DD8DEE95E00E94A839F8016281A5
:10485000CE01C0DD81EF95E00E94A839F8016381A7
:10486000CE01B8DD85EF95E00E94A839F80164819A
:10487000CE01B0DD89EF95E00E94A839F80165818D
:10488000CE01A8DDCE01DF91CF911F910F91ADCF69
:10489000CF92DF92EF92FF92CF93DF93EC0188816A
:1048A0009981AA81BB81181619061A061B0644F0C5
:1048B00081E090E0A0E0B0E088839983AA83BB8385
:1048C0008C819D81AE81BF81181619061A061B06C0
:1048D00044F081E090E0A0E0B0E08C839D83AE8363
:1048E000BF8388859985AA85BB85181619061A067F
:1048F0001B0644F081E090E0A0E0B0E08887998753
:10490000AA87BB878AE095E00E94A83981E994E0F4
:104910000E94A8396091B00A7091B10A8091B20AE0
:104920009091B30A0E94404D6B017C0168817981AE
:104930008A819B810E94404D9B01AC01C701B60159
:104940000E94C94542E00E941B3A81EA94E00E941D
:10495000A8396091B40A7091B50A8091B60A909115
:10496000B70A0E94404D6B017C016C817D818E8174
:104970009F810E94404D9B01AC01C701B6010E947E
:10498000C94542E00E941B3A81EB94E00E94A8399D
:104990006091B80A7091B90A8091BA0A9091BB0AE5
:1049A0000E94404D6B017C01688579858A859B85D5
:1049B0000E94404D9B01AC01C701B6010E94C94550
:1049C00042E00E941B3ACE01DF91CF91FF90EF9021
:1049D000DF90CF900ACF8091820B9091830B892B2F
:1049E00091F58DE090E00E949347FC0114861092AF
:1049F000B00A1092B10A1092B20A1092B30A109241
:104A0000B40A1092B50A1092B60A1092B70A109220
:104A1000B80A1092B90A1092BA0A1092BB0A109200
:104A2000810B1092800B1092AC0A1092AD0A10927A
:104A3000AE0A1092AF0A10922707109226079093A1
:104A4000830B8093820B8091820B9091830B08954E
:104A50000F931F93CF93DF930E94D9088C01C0E07E
:104A6000D0E0BE01C8010E94C118882321F0BE0118
:104A7000C8010E9496082196C13ED10591F78DEF9D
:104A800095E00E94A839A7DFB0DE80E090E0DF91DA
:104A9000CF911F910F9108959EDFFC01148680E055
:104AA00090E00895CF93DF9383E00E94AB0DEC017B
:104AB00092DF91E0CD2B09F490E09093840B82E09B
:104AC0000E94AB0DEC0187DF91E0CD2B09F490E063
:104AD0009093850B8EE00E94AB0DEC017CDF91E0A2
:104AE000CD2B09F490E09093860B8FE00E94AB0DE4
:104AF000EC0171DF91E0CD2B09F490E09093870BEE
:104B000082E10E94AB0DEC0166DF91E0CD2B09F450
:104B100090E09093880B83E10E94AB0DEC015BDF8A
:104B200091E0CD2B09F490E09093890BDF91CF9128
:104B300008952F923F924F925F926F927F928F9241
:104B40009F92AF92BF92CF92DF92EF92FF920F931C
:104B50001F93CF93DF93CDB7DEB72F970FB6F8949F
:104B6000DEBF0FBECDBF9F878E870E94D908EE851E
:104B7000FF85E052FE4F81E04091F4075091F50728
:104B80006091F6077091F707452B462B472B09F4E8
:104B900080E080830E94D908EE85FF85EF51FE4FAB
:104BA00081E04091F8075091F9076091FA07709100
:104BB000FB07452B462B472B09F480E080830E949E
:104BC000D908EE85FF85EE51FE4F81E04091FC074C
:104BD0005091FD076091FE077091FF07452B462B12
:104BE000472B09F480E080830E94D9088091440813
:104BF00090914508A0914608B0914708EE85FF8541
:104C0000ED51FE4F80839183A283B3830E94D90824
:104C10008091480890914908A0914A08B0914B08AA
:104C2000EE85FF85E951FE4F80839183A283B38394
:104C30000E94D90880914C0890914D08A0914E088F
:104C4000B0914F08EE85FF85E551FE4F808391833B
:104C5000A283B3830E94D90880911C0890911D08FB
:104C6000A0911E08B0911F08EE85FF85E550FE4F0C
:104C700080839183A283B3830E94D9088091200806
:104C800090912108A0912208B0912308EE85FF851C
:104C9000E150FE4F80839183A283B3830E94D908A1
:104CA0008091240890912508A0912608B0912708AA
:104CB000EE85FF85ED5FFD4F80839183A283B383F3
:104CC0000E94D90880912C0890912D08A0912E085F
:104CD000B0912F08EE85FF85E95FFD4F80839183BA
:104CE000A283B3830E94D908809130089091310843
:104CF000A0913208B0913308EE85FF85E55FFD4F46
:104D000080839183A283B3830E94D9088091340861
:104D100090913508A0913608B0913708EE85FF854F
:104D2000E15FFD4F80839183A283B3830E94D90802
:104D30008091CC079091CD07A091CE07B091CF077D
:104D4000EE85FF85ED5EFD4F80839183A283B38363
:104D50000E94D9088091D0079091D107A091D207E5
:104D6000B091D307EE85FF85E95EFD4F8083918387
:104D7000A283B3830E94D9088091D4079091D5076C
:104D8000A091D607B091D707EE85FF85E55EFD4F70
:104D900080839183A283B3830E94D908EE85FF8527
:104DA000E15EFD4F81E02091A4073091A5072130FD
:104DB000310509F080E080830E94D908EE85FF85E7
:104DC000E05EFD4F81E02091A8073091A9072130D6
:104DD000310509F080E080830E94D908EE85FF85C7
:104DE000EF5DFD4F81E02091AC073091AD072130A0
:104DF000310509F080E080830E94D908EE85FF85A7
:104E0000E35CFD4F81E040917C0750917D0760910C
:104E10007E0770917F07452B462B472B09F480E0D6
:104E200080830E94D908EE85FF85E25CFD4F81E01A
:104E300040918007509181076091820770918307AC
:104E4000452B462B472B09F480E080830E94D9082C
:104E5000EE85FF85E15CFD4F81E040918407509134
:104E600085076091860770918707452B462B472B56
:104E700009F480E080830E94D908EE85FF85E05C1C
:104E8000FD4F81E020918C0730918D072130310555
:104E900009F080E080830E94D908EE85FF85EF5BF2
:104EA000FD4F81E02091900730919107213031052D
:104EB00009F080E080830E94D908EE85FF85EE5BD3
:104EC000FD4F81E020919407309195072130310505
:104ED00009F080E080830E94D90880915407909166
:104EE0005507A0915607B0915707EE85FF85ED5BFA
:104EF000FD4F80839183A283B3830E94D908809160
:104F0000540790915507A0915607B0915707EE8529
:104F1000FF85E95BFD4F80839183A283B3830E9469
:104F2000D9088091540790915507A0915607B091E8
:104F30005707EE85FF85E55BFD4F80839183A28354
:104F4000B3830E94D908EE85FF85EF5CFD4F81E0B9
:104F500040916407509165076091660770916707FB
:104F6000452B462B472B09F480E080830E94D9080B
:104F7000EE85FF85EE5CFD4F81E040916807509122
:104F8000690760916A0770916B07452B462B472B89
:104F900009F480E080830E94D908EE85FF85ED5CEE
:104FA000FD4F81E040916C0750916D0760916E0755
:104FB00070916F07452B462B472B09F480E08083C7
:104FC0000E94D90880915C0990915D09A0915E09C9
:104FD000B0915F09EE85FF85EE5DFD4F8083918383
:104FE000A283B3830E94D9088091600990916109DE
:104FF000A0916209B0916309EE85FF85EA5DFD4FDE
:1050000080839183A283B3830E94D908809164092D
:1050100090916509A0916609B0916709EE85FF85B9
:10502000E65DFD4F80839183A283B3830E94D908FC
:10503000EE85FF85EC5CFD4F81E02091BC0730914F
:10504000BD072130310509F080E08083EE85FF85C2
:10505000EB5CFD4F1082EE85FF85EA5CFD4F108210
:105060000E94D908EE85FF85E95CFD4F81E0209123
:10507000B8073091B9072130310509F080E080830D
:10508000EE85FF85E85CFD4F1082EE85FF85E75CCD
:10509000FD4F10820E94D908EE85FF85E65CFD4F2A
:1050A00081E02091DC073091DD072130310509F0E6
:1050B00080E080830E94D908EE85FF85E55CFD4F86
:1050C00081E02091E0073091E1072130310509F0BE
:1050D00080E080830E94D908EE85FF85E45CFD4F67
:1050E00081E02091E4073091E5072130310509F096
:1050F00080E080830E94D908EE85FF85E25DFD4F48
:1051000081E020916C0930916D092130310509F061
:1051100080E080830E94D908EE85FF85E15DFD4F28
:1051200081E020917009309171092130310509F039
:1051300080E080830E94D908EE85FF85E05DFD4F09
:1051400081E020917409309175092130310509F011
:1051500080E080830E94D9080E851F85015B1D4F6A
:105160008091040890910508A0910608B091070865
:10517000F80180839183A283B3830E94D908EE84CF
:10518000FF84FDEAEF1AFDEFFF0A80910808909175
:105190000908A0910A08B0910B08F7018083918358
:1051A000A283B3830E94D90880910C0890910D08C6
:1051B000A0910E08B0910F082E853F85295A3D4FCA
:1051C000F90180839183A283B383F80140815181E7
:1051D00062817381141615061606170644F041E025
:1051E00050E060E070E04083518362837383F70195
:1051F00040815181628173811416150616061706C7
:1052000044F041E050E060E070E04083518362830D
:105210007383181619061A061B064CF081E090E0FD
:10522000A0E0B0E0F90180839183A283B383D90128
:105230008D909D90AD90BC90F701C080D180E280B0
:10524000F380D8014D905D906D907C90C4DBFC01A3
:105250004082518262827382C482D582E682F78262
:1052600080869186A286B386EE85FF85E25DFD4F3E
:10527000B081B983EE85FF85EE5DFD4F8081918120
:10528000A281B3814E855F85465C5D4FFA01F08156
:10529000FB834E855F85405C5D4FFA01F081FA83A8
:1052A0004E855F854C5C5D4FFA01F081FF834E8532
:1052B0005F85495C5D4FFA01F081F8874E855F8517
:1052C000435C5D4FFA01F081F987EE85FF85E15E71
:1052D000FD4F2080EE85FF85E052FE4F3080EE8549
:1052E000FF85ED5BFD4F4081518162817381EE85C9
:1052F000FF85ED5EFD4F0081118122813381EE85B6
:10530000FF85E95FFD4FC080D180E280F380EE85AC
:10531000FF85E550FE4F80809180A280B380EE85AE
:10532000FF85ED51FE4F4080518062807380EE8595
:10533000FF8547A250A661A672A683A694A6A5A63D
:10534000B6A6C7A6D0AAE1AAF2AA03AB14AB25ABB6
:1053500036AB47AB50AF61AF72AF33AE24AE2985E9
:1053600025A33A8136A340E450E060E070E0FF9668
:1053700040835183628373832885EE85FF8525AF43
:105380003F8136AFAF014D5B5F4F2B81FA01208328
:10539000EE85FF85EC5BFF4F80839183A283B3830F
:1053A000EE85FF85E85BFF4F39813083AE85BF8591
:1053B00055968D919C9156978633910589F484EF8B
:1053C0009BE0FD01E758FF4F918380833296118265
:1053D000108282EF9BE0369691838083329630C0B4
:1053E0008C33910589F48CEE9BE0EE85FF85E758C0
:1053F000FF4F91838083EE85FF85E558FF4F118233
:1054000010828AEE9BE012C08E97E1F484EE9BE05E
:10541000EE85FF85E758FF4F91838083EE85FF85FA
:10542000E558FF4F118210828EED9BE0EE85FF85DF
:10543000EF57FF4F91838083EE85FF85ED57FF4F38
:1054400011821082EE85FF85838D948D4A97D1F469
:1054500080EF9BE0E358FF4F91838083EE85FF85CB
:10546000E158FF4F118210828EEE9BE0EE85FF85A2
:10547000EB57FF4F91838083EE85FF85E957FF4F00
:1054800011821082EE85FF85E15DFD4F2081298329
:10549000EE85FF85EA5DFD4F40805180628073801C
:1054A000EE85FF85E55CFD4F30813B83EE85FF8512
:1054B000EF5BFD4F9081EE85FF85EB5CFD4F4081FA
:1054C0004F83EE85FF85E85CFD4F50815887EE8560
:1054D000FF85E25CFD4F8081EE85FF85E05EFD4F3C
:1054E0002080EE85FF85EF51FE4F3080EE85FF85F1
:1054F000E95BFD4F20813181428153812A873B87BF
:105500004C875D87EE85FF85E95EFD4F40815181C7
:1055100062817381EE85FF85E55FFD4FC080D1809C
:10552000E280F380EE85FF85E150FE4F8080918020
:10553000A280B380EE85FF85E757FF4F2E853F851C
:1055400029513E4FD9010D911D912D913C91078B11
:10555000108F218F328F838E948EA58EB68EC78E3C
:10556000D0A2E1A2F2A243A354A365A376A32A8505
:105570003B854C855D8527A330A741A752A733A65D
:1055800024A6858B968B80E490E0A0E0B0E087A70E
:1055900090ABA1ABB2AB388535A74F8146A75B81F5
:1055A00053AB44AA55AA66AA77AA898180AF8581A0
:1055B00096818633910589F484EF9BE0AE85BF85A3
:1055C000AE50BF4F8D939C93AE85BF85AC50BF4FFF
:1055D0001D921C9282EF9BE026C08C33910589F4CA
:1055E0008CEE9BE0AE85BF85AE50BF4F8D939C93F4
:1055F000AE85BF85AC50BF4F1D921C928AEE9BE0DA
:1056000012C08E97E1F484EE9BE0AE85BF85AE506C
:10561000BF4F8D939C93AE85BF85AC50BF4F1D92FD
:105620001C928EED9BE0AE85BF85A650BF4F8D933B
:105630009C93AE85BF85A450BF4F1D921C9283855D
:1056400094854A97D9F480EF9BE0EE85FF85EA5078
:10565000FF4F91838083EE85FF85E850FF4F1182D5
:1056600010828EEE9BE0EE85FF85E250FF4F918326
:105670008083EE85FF85F39511821082EE85FF858C
:10568000E05DFD4F908199832E853F85265D3D4FDE
:10569000D9018D919D910D90BC91A02D8B839C8300
:1056A000AD83BE83EE85FF85E45CFD4FB081BA8398
:1056B000EE85FF85EE5BFD4F2080EE85FF85EA5C81
:1056C000FD4F20812F83EE85FF85E75CFD4F308104
:1056D0003887EE85FF85E15CFD4F3080EE85FF85E4
:1056E000EF5DFD4F3081EE85FF85EE51FE4F20814D
:1056F000EE85FF85E55BFD4F80819181A281B381BD
:10570000EE85FF85E55EFD4F4081518162817381A9
:10571000EE85FF85E15FFD4FC080D180E280F380A0
:10572000EE85FF85ED5FFD4F80809180A280B38084
:105730000E851F850E5F1E4FEE85FF85E551FE4FDE
:105740004080518062807380F801478A508E618E5C
:10575000728E838E948EA58EB68EC78ED0A2E1A255
:10576000F2A243A354A365A376A387A390A7A1A7FE
:10577000B2A723A734A7358A268A80E490E0A0E068
:10578000B0E087A790ABA1ABB2AB288525A73F813E
:1057900036A74A8143AB8B819C81AD81BE8184ABAE
:1057A00095ABA6ABB7AB298120AF858196818633B7
:1057B000910589F484EF9BE0EE85FF85E559FE4F66
:1057C00091838083EE85FF85E359FE4F118210821D
:1057D00082EF9BE026C08C33910589F48CEE9BE030
:1057E000EE85FF85E559FE4F91838083EE85FF8529
:1057F000E359FE4F118210828AEE9BE012C08E9711
:10580000E1F484EE9BE0EE85FF85E559FE4F918340
:105810008083EE85FF85E359FE4F118210828EED65
:105820009BE0EE85FF85ED58FE4F91838083EE85EA
:10583000FF85EB58FE4F11821082D8011B968D9187
:105840009C911C974A97E1F480EF9BE0EE85FF85E1
:10585000E159FE4F91838083EE85FF85EF58FE4F1F
:10586000118210828EEE9BE0EE85FF85E958FE4F97
:1058700091838083EE85FF85E758FE4F1182108269
:10588000EE85FF85EF5CFD4F20818E859F854096DC
:10589000222311F053D101C03DD1EE85FF85EE5C8E
:1058A000FD4F20818E859F8587579F4F222311F0C2
:1058B00045D101C02FD1EE85FF85ED5CFD4F808184
:1058C0008823D1F0C8012F960FB6F894DEBF0FBE23
:1058D000CDBFDF91CF911F910F91FF90EF90DF909F
:1058E000CF90BF90AF909F908F907F906F905F9080
:1058F0004F903F902F9022C1C8012F960FB6F89479
:10590000DEBF0FBECDBFDF91CF911F910F91FF90F2
:10591000EF90DF90CF90BF90AF909F908F907F904F
:105920006F905F904F903F902F90F4C02F923F92D6
:105930004F925F926F927F928F929F92AF92BF929F
:10594000CF92DF92EF92FF920F931F93CF93DF934B
:1059500000D000D0CDB7DEB73B011A0129011C836E
:105960000B83FA82E982DE82CD82F4018081882372
:1059700009F474C0F901C080D180E280F38020E096
:1059800030E0A901C701B6010E946B46181674F4F5
:10599000F5012081318142815381C701B6010E9406
:1059A0005D45F2016083718382839383F301E15A41
:1059B000FF4F8081F101008D118DC088D188E28870
:1059C000F388E981FA8180809180A280B380D80138
:1059D000A7019601882341F00E94924E681579052F
:1059E0008A059B0544F023C00E94924E86169706B6
:1059F000A806B906E4F4F20180809180A280B38009
:105A000020E030E04AEF56E4C501B4010E943A4D6F
:105A100087FF0DC020E030E040E85FE3C501B4013E
:105A20000E945E45F2016083718382839383D80173
:105A3000A70196010E94924EE981FA8160837183E9
:105A400082839383F301FD9680819181A281B3814A
:105A5000EB81FC8180839183A283B383ED81FE81FE
:105A600080819181892B49F0C1010E944111F3018C
:105A7000FD96608371838283938326960FB6F89494
:105A8000DEBF0FBECDBFDF91CF911F910F91FF9071
:105A9000EF90DF90CF90BF90AF909F908F907F90CE
:105AA0006F905F904F903F902F900895CF93DF932A
:105AB000EC018CA5882311F061E001C060E08F81CA
:105AC0000E94D30D8DA5882329F08EA5882311F07F
:105AD00061E001C060E08D85DF91CF910C94D30D22
:105AE000CF93DF93EC018CA5882311F060E001C017
:105AF00061E08F810E94D30D8DA5882329F08EA5AA
:105B0000882311F060E001C061E08D85DF91CF91C5
:105B10000C94D30DCF93DF93EC0161E089850E9453
:105B2000D30D8DA5882321F061E08F850E94D30DD0
:105B3000CA59DF4F1882DF91CF910895CF93DF9339
:105B4000EC0160E089850E94D30D8DA5882321F0AA
:105B500060E08F850E94D30DCA59DF4F81E08883B2
:105B6000DF91CF910895CF92DF92EF92FF920F9342
:105B70001F93CF93DF93FC0141AF52AF63AF74AF7C
:105B8000DC01DD964D935D936D937C931397149692
:105B90000D931D932D933C931397EC01CB5BDF4F3B
:105BA000E88283A9882351F083A581114BC037FF78
:105BB00005C01D921D921D921C92139744A955A9D0
:105BC00066A977A9141615061606170634F580ADD2
:105BD000882319F10D911D912D913C911397680126
:105BE000790137FF07C0CC24DD247601C01AD10A21
:105BF000E20AF30A4C155D056E057F0574F437FF64
:105C000007C070956095509541955F4F6F4F7F4FDE
:105C10004D935D936D937C931397DF01A25BBF4F10
:105C20001D921D921D921C921397E25AFF4F81E024
:105C30008083DF91CF911F910F91FF90EF90DF90C4
:105C4000CF90089510161106120613060CF4B1CF6A
:105C5000B5CF0F931F93CF93DF938C01D62FFC0109
:105C6000858981110BC0C8010E949D11C82FC801F0
:105C70000E949011D1110AC08C2F08C0C8010E9447
:105C80009011C82FC8010E949D11F4CFDF91CF91D0
:105C90001F910F910895CF93DF93EC01FC01E85918
:105CA000FF4F81E0808339978081B297882341F04C
:105CB00080819181A281B3810196A11DB11D07C090
:105CC00080819181A281B3810197A109B10980836B
:105CD0009183A283B383FE01E559FF4F2081318177
:105CE000DE01A759BF4FC9019595879520FD03C0D7
:105CF000ED91FC910DC0FE01E80FF91F0190F081BC
:105D0000E02D2D913C91E20FF31F0190F081E02DE9
:105D10008C0F9D1F19958F859889892B11F1FE0194
:105D2000E159FF4F20813181DE01A359BF4FC901E5
:105D30009595879520FD03C0ED91FC910DC0FE0166
:105D4000E80FF91F0190F081E02D2D913C91E20FB9
:105D5000F31F0190F081E02D8C0F9D1FDF91CF91FB
:105D60001994DF91CF9108958F929F92AF92BF9235
:105D7000CF92DF92EF92FF920F931F93CF93DF9317
:105D8000EC01FC01E25BFF4F6081718182819381B4
:105D90000E943E4D6B017C016FA578A989A99AA943
:105DA0000E94404D9B01AC0160E074E284E799E4FD
:105DB0000E94C9454B015C01FE01E65AFF4F60811C
:105DC0007181828193810E943E4D9B01AC01C5018E
:105DD000B4010E94C9454B015C018E010E5A1F4F50
:105DE00020E030E040E05FE30E949F4D9B01AC016A
:105DF000C701B6010E945E450E943F46F8016083DC
:105E0000718382839383CA5ADF4FA5019401C7012E
:105E1000B6010E945E450E943F46688379838A836B
:105E20009B83DF91CF911F910F91FF90EF90DF90B7
:105E3000CF90BF90AF909F908F9008950F931F9336
:105E4000CF93DF93FC01E859FF4F20812223C1F05B
:105E50007A97008111812281338138964081518166
:105E600062817381041715072607370718F1EC01C3
:105E70000E947711CE01DF91CF911F910F9174CFC6
:105E8000FC01E25AFF4F20812223A1F0709700818C
:105E900011812281338134964081518162817381E5
:105EA000041715072607370728F0DF91CF911F91B8
:105EB0000F91F1CEDF91CF911F910F9108952F9205
:105EC0003F924F925F926F927F928F929F92AF928A
:105ED000BF92CF92DF92EF92FF920F931F93CF93D7
:105EE000DF93CDB7DEB762970FB6F894DEBF0FBE73
:105EF000CDBF8C017C0125E4E20EF11CD7018C9111
:105F00009801215A3F4FF801E05AFF4F6F01A80155
:105F1000435C5F4F4A0114971D01882341F0F8014B
:105F200083A5D9018C9381E0F60180832FC0DA012B
:105F30004D915D916D917C91F10180819181A28162
:105F4000B381BB24B394481759076A077B070CF049
:105F5000B12CF901B08277FF07C07095609550951C
:105F600041955F4F6F4F7F4FB7FF07C0B095A0952A
:105F7000909581959F4FAF4FBF4F21E0481759072C
:105F80006A077B070CF420E0D6012C93F4014081D2
:105F9000518162817381411551056105710559F483
:105FA000F801838D948DA58DB68DE65AFF4F8083C1
:105FB0009183A283B383F10180819181A281B38116
:105FC000F80141AC52AC63AC74AC9801225A3F4F1B
:105FD0005901481659066A067B0634F448175907D2
:105FE0006A077B077CF00AC084159505A605B705EE
:105FF0002CF484179507A607B70724F0D7018C91D6
:106000008823D9F0F50180818823B9F0D7018C91DC
:10601000811105C0F701808181110FC006C060E0C9
:10602000C80117DE8111F6CF17C0D6016C9181E04F
:106030006827C8010EDE882379F0D5011C9260E044
:10604000C80107DE882309F4BDC1F801FD9610825E
:10605000118212821382B6C1D80193962D913D917F
:106060004D915C91969729833A834B835C83579635
:106070002D913D914D915C915A972D833E834F8395
:1060800058875B962D913D914D915C915E97298744
:106090003A874B875C87F10180819181A281B3812E
:1060A000F801FD96C080D180E280F380F80141AD17
:1060B00052AD63AD74ADEE59FF4F10823196108230
:1060C0003801F4E66F0E711CF301108298012B5910
:1060D0003F4FF9011082329610824C015D01841A03
:1060E000950AA60AB70AB7FE08C0B094A094909487
:1060F0008094811C911CA11CB11C481759076A0788
:106100007B072CF4C41AD50AE60AF70A04C0C81A99
:10611000D90AEA0AFB0AD501C401B595A795979556
:1061200087958D879E87AF87B88BD801A959BF4FB8
:106130001D01F7FC05C08C149D04AE04BF044CF493
:10614000F801078CF0A1E02DFA8BE98B81E0D901F1
:106150001BC02D853E854F8558892C153D054E0564
:106160005F0508F454C089819A81AB81BC818C158C
:106170009D05AE05BF0564F42D813E812F5F3F4F25
:106180003A8B298B81E0D3018C93F10180839EC0EF
:10619000C701B6010E94404D2B013C0169817A8103
:1061A0008B819C810E94404D9B01AC01C301B201D7
:1061B0000E94C9452B013C016D817E818F819885AC
:1061C00029853A854B855C85621B730B840B950B87
:1061D0000E94404D9B01AC01C301B2010E949F4D42
:1061E0002B013C0169857A858B859C850E94404DF9
:1061F0009B01AC01C301B2010E945E450E94394679
:106200007A8B698B81E0F801EE59FF4F5CC0D501B4
:10621000C40129813A814B815C81821B930BA40BC1
:10622000B50BC816D906EA06FB065CF42D813E8143
:106230002E5F3F4F3A8B298B81E0F801EC59FF4FDD
:1062400042C0C501B4016C197D098E099F090E94E5
:10625000404D2B013C0169817A818B819C810E9498
:10626000404D9B01AC01C301B2010E94C9452B0105
:106270003C016D817E818F81988529853A854B858A
:106280005C85621B730B840B950B0E94404D9B0138
:10629000AC01C301B2010E949F4D2B013C016985F5
:1062A0007A858B859C850E94404D9B01AC01C30182
:1062B000B2010E945E450E9439467A8B698B81E06B
:1062C000F801ED59FF4F8083D1018C93F80184814F
:1062D0008823B1F00E94560FD80112964D905C9021
:1062E0001397052C000C66087708DC01CB01841994
:1062F0009509A609B709893E9340A105B10568F43F
:10630000F801E65AFF4F29893A89C901A0E0B0E0B7
:1063100080839183A283B38392CE0E94560FD801CB
:1063200013967C936E9312978EE494E00E94A839A2
:1063300081E096E00E94A83960E070E0CB010E9405
:10634000F43987E096E00E94A839C701B6010E949F
:10635000F4398DE096E0FCD7C501B4010E94F43910
:1063600083E196E0F5D74AE06D857E858F85988933
:10637000F0D78AE196E0ECD769817A818B819C81A4
:106380000E94F43980E296E0E3D769857A858B85AF
:106390009C850E94F43986E296E0DAD76D817E8191
:1063A0008F8198850E94F4398CE296E0D1D782E8FB
:1063B00094E0CED789899A890E94EA3A86EC93E0E4
:1063C000C7D79ECF62960FB6F894DEBF0FBECDBF83
:1063D000DF91CF911F910F91FF90EF90DF90CF90C1
:1063E000BF90AF909F908F907F906F905F904F90F5
:1063F0003F902F9008950F931F93FC01EB5BFF4F8D
:106400002081211110C038970081118122813381B0
:1064100034964081518162817381041715072607E4
:10642000370744F404C0FC0123A5222319F01F916F
:106430000F9156CB1F910F9139CBFC011382128221
:10644000148216821582108617821286118614868F
:10645000138616861586108A1786128A118A148A60
:10646000138ADC01A25ABF4F1C9211AE12AE13AEBA
:1064700014AE91971D921D921D921C921397149623
:106480001D921D921D921C92139714961C925A965F
:106490001C9211961C9212961C9211961C921196A7
:1064A0001C9211961C9211961C9211961C92119698
:1064B0001C92119683ED9EE011969C938E931296FA
:1064C00011961C921E9212968FEC9EE011969C9350
:1064D0008E93129611961C921E9212968BEC9EE051
:1064E00011969C938E93129611961C921E92129660
:1064F00087EC9EE08D939C93E958FF4F11821082A8
:1065000008950E94EB240C9452250E94EB240C94D5
:106510000724CF93DF93EC01FC01EA54FD4F108276
:10652000E558F1098081811103C0CE014096F2DA6D
:10653000FE01EE5CFD4F8081811104C0CE018757C2
:106540009F4FE8DAFE01ED5CFD4F8081811104C0B0
:10655000CE018E5F9E4FDEDA64E670E080E090E070
:10656000DF91CF910C941E0F2F923F924F925F922A
:106570006F927F928F929F92AF92BF92CF92DF9253
:10658000EF92FF920F931F93CF93DF93EC010E9442
:10659000D908FE01EB57FD4F8091E4089091E50882
:1065A000918380830E94D908FE01E957FD4F8091B5
:1065B000E8089091E908918380830E94D908FE0140
:1065C000E757FD4F8091EC089091ED08918380830F
:1065D0000E94D9088E0105571D4F60910C097091DA
:1065E0000D0980910E0990910F090E94404DF8010C
:1065F00060837183828393830E94D9081E01F1E72F
:106600002F1AFDEF3F0A60911009709111098091D6
:106610001209909113090E94404DF101608371832A
:10662000828393830E94D90820E030E048EC52E452
:10663000F80160817181828193810E94C9452B019B
:106640003C0120E030E048EC52E4F10160817181CE
:10665000828193810E94C9454B015C0160911409BC
:106660007091150980911609909117090E94404D6B
:1066700020E030E048EC52E40E94C9456B017C0107
:106680002AE037ED43E25CE3C301B2010E946B46AE
:1066900018168CF420E030E046EC52E4C301B2015D
:1066A0000E943A4D87FD0FC0412C512C46EC642EC0
:1066B00042E4742E08C05AE0452E57ED552E53E2A1
:1066C000652E5CE3752EF8014082518262827382EE
:1066D0002AE037ED43E25CE3C501B4010E946B465A
:1066E00018168CF420E030E046EC52E4C501B40109
:1066F0000E943A4D87FD0FC0812C912C26ECA22ED2
:1067000022E4B22E08C03AE0832E37ED932E33E216
:10671000A32E3CE3B32EF10180829182A282B38248
:106720002AE037ED43E25CE3C701B6010E946B4605
:1067300018168CF420E030E046EC52E4C701B601B4
:106740000E943A4D87FD0FC0C12CD12C86ECE82E5B
:1067500082E4F82E08C09AE0C92E97EDD92E93E274
:10676000E92E9CE3F92EFE01ED56FD4FC082D18249
:10677000E282F3820E94D9088091CC089091CD08E2
:10678000FE01E656FD4F918380830E94D9088091D7
:10679000D0089091D108FE01E456FD4F918380838B
:1067A0000E94D9088091D4089091D508FE01E25644
:1067B000FD4F918380830E94D9088091F4089091C5
:1067C000F508FE01E056FD4F918380830E94D908B1
:1067D0008091F8089091F908FE01EE55FD4F9183E4
:1067E00080830E94D9088091FC089091FD08FE01E9
:1067F000EC55FD4F918380830E94D90880911C093C
:1068000090911D09FE01EA55FD4F918380830E94FE
:10681000D9088091200990912109FE01E855FD4F8A
:10682000918380830E94D908809124099091250941
:10683000FE01E655FD4F918380830E94D908809127
:10684000340990913509FE01E455FD4F9183808311
:106850000E94D9088091380990913909FE01E255CA
:10686000FD4F918380830E94D90880913C099091CB
:106870003D09FE01E055FD4F918380830E94D908B8
:106880008091BC089091BD08A091BE08B091BF084E
:10689000FE01E956FD4F0197A105B10519F481E00C
:1068A000808301C010820E94D9088091C008909115
:1068B000C108A091C208B091C308FE01E856FD4F7F
:1068C0000197A105B10519F481E0808301C0108210
:1068D0000E94D9088091C4089091C508A091C6086B
:1068E000B091C708C756DD4F0197A105B10519F44E
:1068F00081E0888301C01882DF91CF911F910F91B1
:10690000FF90EF90DF90CF90BF90AF909F908F90CF
:106910007F906F905F904F903F902F9008952F92AF
:106920003F924F925F926F927F928F929F92AF921F
:10693000BF92CF92DF92EF92FF920F931F93CF936C
:10694000DF93CDB7DEB7AB970FB6F894DEBF0FBEBF
:10695000CDBF9BA78AA71B010E9499258AA59BA54D
:1069600003DE8AA59BA5CDDD8AA59BA5CEDD21E012
:1069700022163104C9F132E02316310409F466C04D
:106980002114310409F094C04AA45BA440E1440EF0
:10699000511C8AA59BA585589E4F9A878987EAA591
:1069A000FBA5E35CFD4F90819B8BAAA5BBA5A55AD7
:1069B000BD4FBC87AB87EAA5FBA5EB57FD4FFD8B11
:1069C000EC8B2AA53BA529563D4F398F288F4AA528
:1069D0005BA546525E4F5A8B498B8DE890E09F8BAA
:1069E0008E8BA5E1B0E061C04AA45BA4B9E84B0E70
:1069F000511CEAA5FBA5EB56FE4FFA87E987EAA5ED
:106A0000FBA5E25CFD4F20812B8B4AA55BA5415A7B
:106A10005D4F5C874B878AA59BA589579D4F9D8BB2
:106A20008C8BAAA5BBA5A856BD4FB98FA88FEAA588
:106A3000FBA5E452FE4FFA8BE98B2EE830E03F8B4A
:106A40002E8B46E150E05E834D8335C04AA45BA4A3
:106A50005EEF451A550A8AA59BA581559E4F9A87D8
:106A60008987EAA5FBA5E15CFD4F90819B8BAAA5D8
:106A7000BBA5AD59BD4FBC87AB87EAA5FBA5E757C2
:106A8000FD4FFD8BEC8B2AA53BA527563D4F398F3B
:106A9000288F4AA55BA542525E4F5A8B498B8FE8DF
:106AA00090E09F8B8E8BA7E1B0E0BE83AD8303C0E7
:106AB00082E396E00CC0C2010E949D11811105C0C5
:106AC000C2010E949011882331F083EC96E040D4FB
:106AD00081E090E0DAC38EE494E03AD481E696E077
:106AE00037D4D2018C9175D489EF96E031D486ECFD
:106AF00093E02ED481E090E0E989FA899183808344
:106B00000AA51BA506521E4FD8014D915C91B201FA
:106B10008AA59BA50E944915C20110D8F20183A540
:106B20009201215A3F4F3901882339F0C2010E9456
:106B3000702D81E0F301808305C0C2010E94562DB3
:106B4000D3011C9289859A850E944111F201FD961C
:106B50006083718382839383EB85FC85108211822D
:106B600012821382EAA5FBA5E55AFD4F108211821D
:106B700012821382EAA5FBA5E15AFD4F1082118211
:106B800012821382EAA5FBA5ED59FD4F10821182F6
:106B90001282138286E090E0A989BA898D939C9332
:106BA000F80140815181B2018AA59BA50E94491537
:106BB00041E050E0B2018AA59BA50E942C1521E07E
:106BC00030E040E050E02D873E874F87588BC10171
:106BD00089569D4F4AA55BA5480F591F5B8F4A8F69
:106BE000C101880F991F880F991F9A838983855740
:106BF0009D4FAAA5BBA5A80FB91FBF8FAE8FC1011E
:106C00008D5A9E4F880F991FEAA5FBA5E80FF91F23
:106C1000F9A3E8A389819A8187589D4F2AA53BA5AE
:106C2000280F391F3BA32AA389819A8183599D4F3D
:106C30004AA55BA5480F591F5DA34CA389819A8182
:106C4000855A9D4FAAA5BBA5A80FB91FBFA3AEA388
:106C500069807A80EAA5FBA56E0E7F1EF9EF6F1A98
:106C6000FDEF7F0A8A8C9B8CAE8CBF8CC8A0D9A00C
:106C7000EAA0FBA00CA11DA12EA13FA149855A8528
:106C8000B2018AA59BA50E94962C8AE89BE00E94EF
:106C90005F0A1816190624F01C821B8210E010C02F
:106CA0008AE89BE00E943D0A8F7D85349105A1F71B
:106CB00089EE94E04DD321E030E03C832B8311E05A
:106CC000C2010E949D1181111DC0C2010E9490113C
:106CD000811118C0111116C0AC89BD896D917C91CC
:106CE000072E000C880B990B0E94404D9B01AC01B4
:106CF000EB85FC8560817181828193810E943A4D90
:106D000087FD6AC281EA96E023D3C2010E949011F6
:106D100081115FC242E050E0B2018AA59BA50E94AA
:106D20002C158EE494E014D381E696E011D3D201C1
:106D30008C914FD388E696E00BD386EC93E008D392
:106D4000EB81FC81EF2BD1F48BE796E001D382E855
:106D500094E0FED28FEB94E0FBD28D819E813AD4F9
:106D600082E894E0F5D281EC94E0F2D2FB898F2F97
:106D700090E030D40E94EB240E94F5238AA59BA5C5
:106D8000C0DB8AA59BA5C1DB8EE494E0E1D281E65D
:106D900096E0DED2D2018C911CD38FE796E0D8D258
:106DA00086EC93E0D5D2EB85FC85108211821282AD
:106DB0001382D2019B968C918201015A1F4F882326
:106DC00031F0C2010E94562DF801108206C0C201A6
:106DD0000E94702D81E0D8018C9389859A850E944C
:106DE0004111F201FD966083718382839383EAA54A
:106DF000FBA5E55AFD4F1082118212821382EAA58B
:106E0000FBA5E15AFD4F1082118212821382EAA57E
:106E1000FBA5ED59FD4F10821182128213828985E4
:106E20009A850E9441116A8F7B8F8C8F9D8F21E004
:106E300030E040E050E02D833E834F835887C1010E
:106E400089569D4F4AA55BA5480F591F5F8F4E8FEE
:106E500089819A8185579D4FAAA5BBA5A80FB91F07
:106E6000B9A3A8A3C1018D5A9E4F880F991FEAA507
:106E7000FBA5E80FF91FFBA3EAA389819A81875834
:106E80009D4F2AA53BA5280F391F3DA32CA389811F
:106E90009A8183599D4F4AA55BA5480F591F5FA34F
:106EA0004EA389819A81855A9D4FAAA5BBA5A80F9B
:106EB000B91FB9A7A8A7AD81BE811197BE87AD87BD
:106EC0003D01EB81FC81EF2B09F0C6C08E8C9F8CBD
:106ED000A8A0B9A0CAA0DBA0ECA0FDA00EA11FA194
:106EE00028A539A549855A85B2018AA59BA50E9486
:106EF000962C8AE89BE00E945F0A1816190614F087
:106F000010E010C08AE89BE00E943D0A8F7D853426
:106F10009105B1F789EE94E01BD2E1E0F0E0FC834B
:106F2000EB8311E02D853E852A30310538F4AB85A1
:106F3000BC851D921D921D921C921397BB89C201A4
:106F4000B1119EC10E949011811182C0112319F0CC
:106F50006D847E847DC0EC89FD8960817181072EFE
:106F6000000C880B990B0E94404D9B01AC01AB8536
:106F7000BC856D917D918D919C910E943A4D87FFCA
:106F8000E7CFC2010E944B2E69807A80EAA5FBA55B
:106F90006E0E7F1EF9EF6F1AFDEF7F0AD3012D9160
:106FA0003D914D915C9160E573EC80E090E00E9432
:106FB0006C4EC9010E94130FF3012081318142817F
:106FC0005381A3E0B0E00E94884E9B01AC016D812B
:106FD0007E818F8198850E946C4E672B682B692B70
:106FE00099F486E493E0B4D10E94EB240E94F52347
:106FF0008EE494E0ADD183E996E0AAD18D819E81A3
:10700000E9D286EC93E0A4D1C2010E947711E98114
:10701000FA812AA53BA5E20FF31FE95FFD4F20810E
:1070200031814281538160E573EC80E090E00E9401
:107030006C4EC9010E94130F8D819E81AF81B8856E
:107040000196A11DB11D8D839E83AF83B88733CF79
:1070500081EA96E07DD104C021E030E03C832B83BF
:107060008EE494E075D181E696E072D1D2018C91E4
:10707000B0D185EB96E06CD186EC93E069D189853F
:107080009A850E944111E88DF98DEF2BA1F0DC016A
:10709000CB012A8D3B8D4C8D5D8D821B930BA40BF8
:1070A000B50BB7FF07C0B095A095909581959F4F00
:1070B000AF4FBF4F3C014B815C81452BF9F48BE70F
:1070C00096E046D182E894E043D18FEB94E040D142
:1070D0008E899F897FD282E894E03AD181EC94E056
:1070E00037D1B301072C000C880B990B0E94404D3F
:1070F00042E0A1D10E94EB240E94F52385E090E0BC
:10710000A989BA898D939C930AA51BA506521E4F87
:10711000F80140815181B2018AA59BA50E944915C1
:10712000C2010E948A2D8AA59BA5EBD98AA59BA5A1
:10713000ECD9F1E02F163104A9F022E02216310437
:1071400001F1232861F50E94EB24C301770CAA0BFF
:10715000BB0B8093B00A9093B10AA093B20AB0938C
:10716000B30A1DC00E94EB24C301770CAA0BBB0B12
:107170008093B40A9093B50AA093B60AB093B70A65
:107180000EC00E94EB24C301770CAA0BBB0B8093AB
:10719000B80A9093B90AA093BA0AB093BB0A0E94A6
:1071A000EB240E944824A989BA891D921C92F801F7
:1071B00040815181B2018AA59BA50E94491540E0FA
:1071C00050E0B2018AA59BA50E942C158B819C8161
:1071D0005CC031E03B8B9ECDC2010E944B2ED3019F
:1071E0002D913D914D915C9160E573EC80E090E0D4
:1071F0000E946C4EC9010E94130FF301208131815E
:1072000042815381A3E0B0E00E94884E9B01AC0113
:107210006D857E858F8598890E946C4E672B682BC3
:10722000692B39F486E493E093D00E94EB240E940A
:10723000F523C2010E947711D3012D913D914D910B
:107240005C9160E573EC80E090E00E946C4EC901B7
:107250000E94130F2D853E854F8558892F5F3F4F24
:107260004F4F5F4F2D873E874F87588B4B815C81F7
:10727000452B09F4F7CC81E090E09C838B834ACDC9
:107280000E949D11811164CE61CEAB960FB6F89429
:10729000DEBF0FBECDBFDF91CF911F910F91FF9049
:1072A000EF90DF90CF90BF90AF909F908F907F90A6
:1072B0006F905F904F903F902F900895CF93DF9302
:1072C000FC01E353FE4F408151814115510559F1B5
:1072D000EC01CF52DE4F2881398187539E4F24170E
:1072E0003507C8F4FC0180819181009761F0FC01B1
:1072F000E20FF31F80818A3041F08D3029F486EC53
:1073000093E026D002C080E064D088819981019604
:107310009983888308C040E050E068EC73E00E94E5
:107320000E0D19821882DF91CF910895009769F0B0
:10733000FC0101900020E9F73197AF01481B590B80
:10734000BC018AE89BE00C94120A80E090E008956A
:10735000EDCF8F929F92AF92BF920F931F93CF93D7
:10736000DF93CDB7DEB7A1970FB6F894DEBF0FBE9F
:10737000CDBF19A2423008F44AE08E010F5D1F4FC5
:10738000842E912CA12CB12CA50194010E94984E21
:10739000E62FB901CA0101501109EA3014F4E05D89
:1073A00001C0E95CD801EC93232B242B252B61F73A
:1073B000C801BCDFA1960FB6F894DEBF0FBECDBFEB
:1073C000DF91CF911F910F91BF90AF909F908F90C1
:1073D0000895E0918A0BF0918B0B0190F081E02DE4
:1073E000682F8AE89BE01994CF92DF92EF92FF9288
:1073F000CF93DF9397FF17C06B017C018DE2E9DF2C
:10740000EC0166277727CB016C197D098E099F094E
:107410004AE09FDF8C0F9D1FDF91CF91FF90EF908F
:10742000DF90CF9008954AE0DF91CF91FF90EF90E9
:10743000DF90CF908ECF4F925F926F927F928F921C
:107440009F92AF92BF92CF92DF92EF92FF926B0129
:107450007C01B42E9B01AC010E946F46882319F079
:1074600088E197E027C026013701E89477F82FEFED
:107470003FEF4FE75FE7C301B2010E946F46811102
:107480000DC02FEF3FEF4FE75FE7C301B2010E944E
:107490003A4D18161CF48CE197E00CC02FEF3FEF2B
:1074A0004FE75FE4C701B6010E946B4618167CF4F3
:1074B00080E297E0FF90EF90DF90CF90BF90AF9089
:1074C0009F908F907F906F905F904F902FCF2FEF76
:1074D0003FEF4FE75FECC701B6010E943A4D87FDD1
:1074E000E7CF20E030E0A901C701B6010E943A4D84
:1074F00087FF08C08DE26DDF4C01F7FAF094F7F8D2
:10750000F09402C0812C912CA12C60E070E080E00E
:107510009FE3AB1441F020E030E040E251E40E94F0
:10752000C945A394F6CF9B01AC01C701B6010E94E7
:107530005E452B013C010E943F466B017C010E948D
:107540003E4D9B01AC01C301B2010E945D452B0180
:107550003C014AE0C701B601FCDE7C01E80CF91CE5
:10756000BB2021F08EE235DFE80EF91EDB2CDD209A
:1075700019F120E030E040E251E4C301B2010E9481
:107580009F4D2B013C010E943F464B01A12CB12C89
:107590004AE0C501B401DDDEE80EF91EC501B40103
:1075A0000E943E4D9B01AC01C301B2010E945D45AA
:1075B0002B013C01DA94DBCFC701FF90EF90DF9005
:1075C000CF90BF90AF909F908F907F906F905F9083
:1075D0004F900895BC01990F880B990B05CF7894B3
:1075E00084B5826084BD84B5816084BD85B58260C8
:1075F00085BD85B5816085BD80916E008160809379
:107600006E001092810080918100826080938100E1
:1076100080918100816080938100809180008160F1
:10762000809380008091B10084608093B10080914C
:10763000B00081608093B00080919100826080935F
:1076400091008091910081608093910080919000E1
:107650008160809390008091A10082608093A1005E
:107660008091A10081608093A1008091A000816041
:107670008093A000809121018260809321018091FC
:10768000210181608093210180912001816080939C
:10769000200180917A00846080937A0080917A0042
:1076A000826080937A0080917A00816080937A0072
:1076B00080917A00806880937A001092C10061E026
:1076C00086E30E94D70E61E087E30E94D70E61E057
:1076D00086E20E94D70E61E08AE10E94D70E61E047
:1076E0008CE10E94D70E61E088E10E94D70E62E033
:1076F00083E00E94D70E62E082E00E94D70E62E033
:1077000080E10E94D70E62E081E10E94D70E62E024
:107710008FE10E94D70E62E081E20E94D70E61E005
:107720008CE30E94D70E61E08DE30E94D70E61E0EA
:1077300088E30E94D70E62E08EE00E94D70E62E0DE
:107740008FE00E94D70E62E087E10E94D70E62E0D0
:1077500089E10E94D70E62E083E20E94D70E62E0C8
:1077600085E20E94D70E61E08EE20E94D70E61E0B2
:1077700080E30E94D70E61E08EE30E94D70E62E0A4
:1077800082E10E94D70E62E083E10E94D70E62E0A0
:107790008BE10E94D70E62E08DE10E94D70E62E07D
:1077A00087E20E94D70E62E089E20E94D70E61E074
:1077B0008AE00E94D70E61E088E00E94D70E61E067
:1077C00089E00E94D70E61E08DE00E94D70E62E052
:1077D0008FE30E94D70E62E08BE30E94D70E62E037
:1077E00088E20E94D70E62E080E40E94D70E62E039
:1077F0008AE20E94D70E62E08CE20E94D70E62E01D
:1078000081E40E94D70E62E082E40E94D70E62E01B
:1078100084E30E94D70E62E085E30E94D70E62E007
:1078200080E00E94D70E62E081E00E94D70E62E005
:1078300089E30E94D70E62E08AE30E94D70E62E0DD
:1078400081E30E94D70E62E082E30E94D70E62E0DD
:1078500083E30E94D70E62E08BE20E94D70E62E0C3
:107860008DE20E94D70E62E08FE20E94D70E62E0A6
:1078700080E20E94D70E61E086E20E94D30D61E0B3
:1078800088E10E94D30D61E088E30E94D30D61E09E
:107890008EE30E94D30DE0919A0BF0919B0B82E056
:1078A0008083E091960BF091970B1082E091980BFA
:1078B000F091990BD0E1D0831092A20BE0919E0B36
:1078C000F0919F0B86E08083E0919C0BF0919D0BE3
:1078D000808180618083E0919C0BF0919D0B808181
:1078E00088608083E0919C0BF0919D0B8081806883
:1078F0008083E0919C0BF0919D0B80818F7D808334
:1079000064E670E080E090E00E941E0F0E949016F6
:107910000E94F8110E94D9160E94A9160E94560FC3
:107920006093600B7093610B8093620B9093630B79
:107930008FE19CE09093250780932407C1E0C093DA
:107940006F00D093810010928000C093BE0A80E047
:1079500092E09093BD0A8093BC0A90938700809335
:10796000860081E180938100109281001092850051
:10797000109284008091BE0A8061809381000E94F1
:10798000560F60935C0B70935D0B80935E0B90932E
:107990005F0B0E94560F6093640B7093650B80938E
:1079A000660B9093670B0E94560F6093600B709369
:1079B000610B8093620B9093630B0E94D9088091B6
:1079C000780790917907A0917A07B0917B0701978A
:1079D000A105B105E1F482E693E0BADC0E949016BD
:1079E000CF931F921F921F921F92812C912CA12C3A
:1079F000B12CC12CD12C760197018601B701A601CB
:107A00000E9457190F900F900F900F900F900E94A7
:107A1000D9088091740790917507A0917607B0916D
:107A200077070197A105B105E9F48AE793E090DCB7
:107A30000E9490161F9221E02F931F921F921F9277
:107A4000812C912CA12CB12CC12CD12C7601970129
:107A50008601B701A6010E9457190F900F900F9051
:107A60000F900F900E94D908809170079091710734
:107A7000A0917207B09173070197A105B105E9F4D0
:107A800082E993E065DC0E9490161F921F9221E02C
:107A90002F931F921F92812C912CA12CB12CC12CC1
:107AA000D12C760197018601B701A6010E945719D2
:107AB0000F900F900F900F900F908AEA93E048DCA0
:107AC0000E94560F6093640B7093650B8093660B56
:107AD0009093670B0091600B1091610B2091620BEA
:107AE0003091630B601771078207930748F4609326
:107AF000600B7093610B8093620B9093630B2CC0AF
:107B0000DC01CB01801B910BA20BB30B883E934091
:107B1000A105B10508F108511C4F2F4F3F4F0093AD
:107B2000600B1093610B2093620B3093630B0E94E8
:107B3000D916EC010E947818CE010C960E94781894
:107B4000CE0148960E947818CE0184960E9478183B
:107B5000CE01C0960E9478188AE89BE00E945F0AD6
:107B6000892B09F49CC50E94560F60935C0B70939F
:107B70005D0B80935E0B90935F0B8AE89BE00E9405
:107B80003D0A80935B0B982F9F7D953479F020916F
:107B9000590B30915A0BF901E95DF44F80832F5F47
:107BA0003F4F30935A0B2093590B06C00E94EB2491
:107BB00021E0DC011C962C938091590B90915A0B7B
:107BC0008133910564F02AE020935B0BFC01E95DB1
:107BD000F44F2083019690935A0B8093590B809118
:107BE0005B0B2091590B30915A0B8A3039F4C90143
:107BF0000197A4EFBAE0E7E2FBE004C022333105CD
:107C0000B4F74DC5AF0147525B40481759071CF404
:107C100041914D93F7CFFC01EC50F54F108222308B
:107C200031050CF438C58DE093E092DB82E894E0F6
:107C30008FDB89EC93E08CDB84EF9AE089DB89ECC5
:107C400093E086DB86EC93E083DB8AE390E00E949E
:107C500093478C01FC0112821382148215821682D2
:107C6000178210861186128613861486158616864C
:107C70001786108A118A128A138A148A158A168A1C
:107C8000178A108E118E128E138E148E158E168EEC
:107C9000178E10A211A212A213A214A215A216A24C
:107CA00017A210A611A612A613A614A615A616A60C
:107CB00017A610AA11AA12AA13AA14AA15AA16AADC
:107CC00017AA10AE11AE6CE072E084EF9AE00E9449
:107CD000C348EC0188818654823010F10E94D90893
:107CE00040903C0750903D0760903E0770903F07E2
:107CF000F801C6A8D7A8E0ACF1AC0E94EB24C09272
:107D0000AC0AD092AD0AE092AE0AF092AF0AC091EE
:107D10000002D0910102C230D10508F4FEC1F1C1C8
:107D20006BEC73E0CE010E946447892B09F4D3C049
:107D30006EEC73E0CE010E946447892B09F4CBC03E
:107D400062ED73E0CE010E946447892B09F4C6C03E
:107D500065ED73E0CE010E946447892B09F4BEC033
:107D600069ED73E0CE010E946447892B09F4B9C024
:107D70006DED73E0CE010E946447892B09F4B4C015
:107D800061EE73E0CE010E946447892B09F4ACC018
:107D900064EE73E0CE010E946447892B09F4A7C00A
:107DA00068EE73E0CE010E946447892B09F4A2C0FB
:107DB0006CEE73E0CE010E946447892B09F49DC0EC
:107DC00060EF73E0CE010E946447892B09F498C0EC
:107DD00064EF73E0CE010E946447892B09F493C0DD
:107DE00068EF73E0CE010E946447892B09F48EC0CE
:107DF0006CEF73E0CE010E946447892B09F489C0BF
:107E000060E074E0CE010E946447892B09F484C0CD
:107E100064E074E0CE010E946447892B09F47FC0BE
:107E200068E074E0CE010E946447892B09F47AC0AF
:107E30006CE074E0CE010E946447892B09F475C0A0
:107E400060E174E0CE010E946447892B09F470C0A0
:107E500064E174E0CE010E946447892B09F46BC091
:107E600068E174E0CE010E946447892B09F466C082
:107E70006CE174E0CE010E946447892B09F461C073
:107E800060E274E0CE010E946447892B09F45CC073
:107E900064E274E0CE010E946447892B09F457C064
:107EA00068E274E0CE010E946447892B09F452C055
:107EB0006CE274E0CE010E946447892B09F44DC046
:107EC00060E374E0CE010E946447892B09F448C046
:107ED0008FEF9FEF47C080E090E044C081E090E0EA
:107EE00041C08CE190E03EC08DE690E03BC08FE663
:107EF00090E038C080E790E035C081E790E032C084
:107F000082E790E02FC083E790E02CC084E790E008
:107F100029C088E790E026C089E790E023C08AE77F
:107F200090E020C083E890E01DC084E890E01AC093
:107F30008DE890E017C08EE890E014C08FE890E0E4
:107F400011C080E990E00EC081EA90E00BC085EBA3
:107F500090E008C086EB90E005C087EB90E002C09F
:107F600088EB90E09093010280930002209709F43F
:107F7000B5CE8881883559F4CE0101960E94C0485B
:107F8000D80112966D937D938D939C93159788815C
:107F9000893549F4CE0101960E94C048F8016683F4
:107FA00077838087918788818A3559F4CE0101963D
:107FB0000E94C048D8011A966D937D938D939C932F
:107FC0001D978881813451F4CE0101960E94C048EA
:107FD00050D6F80166877787808B918B88818234B1
:107FE00061F4CE0101960E94C04843D6D801529652
:107FF0006D937D938D939C9355978881833451F431
:10800000CE0101960E94C04834D6F801668B778B6A
:10801000808F918F8881833559F4CE0101960E941B
:10802000C048D8015A966D937D938D939C935D972C
:108030008881803551F4CE0101960E94C04819D63E
:10804000F801668F778F80A391A38881863561F4CC
:10805000CE0101960E94C0480CD6D80192966D932D
:108060007D938D939C9395978881873551F4CE01AC
:1080700001960E94C048FDD5F80166A377A380A7AA
:1080800091A78881853461F4CE0101960E94C04891
:10809000F0D5D8019A966D937D938D939C939D977F
:1080A0008881843551F4CE0101960E94C048E1D503
:1080B000F80166A777A780AB91AB88818D3461F416
:1080C000CE0101960E94C048D4D5D801D2966D93B6
:1080D0007D938D939C93D5978881813551F4CE0102
:1080E00001960E94C048C5D5F80166AB77AB80AF5A
:1080F00091AF64E374E080E090E00E94C348EC013B
:1081000035CFCE018F569109DD24D394059738F0F1
:10811000C437D10521F0D12C02C0DD24D3940E94B4
:10812000EB24DC011C968C91882381F0CD36D1059F
:1081300009F42AC4CE01885791098330910548F18A
:10814000CD97039730F181E093E09DC201151105B1
:1081500019F48DEF92E097C2CF3FBFEFDB07C9F371
:108160002097D1F48091BF0A9091C00A892B61F4C5
:1081700082E090E0D8D625E132E0FC013183208313
:108180009093C00A8093BF0AE090BF0AF090C00AA3
:1081900053C001151105E9F2CC31D105B9F4809134
:1081A000C10A9091C20A892B61F482E090E0BBD6AB
:1081B0002FE132E0DC012D933C939093C20A80932F
:1081C000C10AE090C10AF090C20A6AC0CD36D1055A
:1081D000B9F48091C30A9091C40A892B61F482E0BA
:1081E00090E0A1D629E232E0FC0131832083909314
:1081F000C40A8093C30AE090C30AF090C40A50C036
:10820000CF36D105B9F48091C50A9091C60A892B61
:1082100061F482E090E087D623E332E0DC012D9325
:108220003C939093C60A8093C50AE090C50AF090EB
:10823000C60A50C0E12CF12CC037D105B9F48091A9
:10824000C70A9091C80A892B61F482E090E06BD64E
:108250002DE332E0FC01318320839093C80A8093A0
:10826000C70AE090C70AF090C80A68C0C137D105B4
:10827000B9F48091C90A9091CA0A892B61F482E00D
:1082800090E051D627E432E0DC012D933C939093AB
:10829000CA0A8093C90AE090C90AF090CA0A68C065
:1082A000C237D105B9F48091CB0A9091CC0A892BC1
:1082B00061F482E090E037D621E532E0FC013183C1
:1082C00020839093CC0A8093CB0AE090CB0AF09065
:1082D000CC0A68C0C337D105B9F48091CD0A90911A
:1082E000CE0A892B61F482E090E01DD62BE532E0C6
:1082F000DC012D933C939093CE0A8093CD0AE090BD
:10830000CD0AF090CE0A68C0C437D105B9F4809187
:10831000CF0A9091D00A892B61F482E090E003D6D5
:1083200025E632E0FC01318320839093D00A8093CC
:10833000CF0AE090CF0AF090D00A68C0C837D105C4
:10834000B9F48091D10A9091D20A892B61F482E02C
:1083500090E0E9D52FE632E0DC012D933C93909339
:10836000D20A8093D10AE090D10AF090D20A68C074
:10837000C937D105B9F48091D30A9091D40A892BD9
:1083800061F482E090E0CFD529E732E0FC0131834F
:1083900020839093D40A8093D30AE090D30AF0907C
:1083A000D40A68C0CA37D105B9F48091D50A909132
:1083B000D60A892B61F482E090E0B5D523E832E05B
:1083C000DC012D933C939093D60A8093D50AE090DC
:1083D000D50AF090D60A68C0CD38D105B9F480919D
:1083E000D70A9091D80A892B61F482E090E09BD55E
:1083F0002DE832E0FC01318320839093D80A8093EA
:10840000D70AE090D70AF090D80A68C0CE38D105D4
:10841000B9F48091D90A9091DA0A892B61F482E04B
:1084200090E081D527E932E0DC012D933C939093D5
:10843000DA0A8093D90AE090D90AF090DA0A68C083
:10844000CF38D105B9F48091DB0A9091DC0A892BF1
:1084500061F482E090E067D521EA32E0FC013183EB
:1084600020839093DC0A8093DB0AE090DB0AF09093
:10847000DC0A68C0C039D105B9F48091DD0A909159
:10848000DE0A892B61F482E090E04DD52BEA32E0E0
:10849000DC012D933C939093DE0A8093DD0AE090FB
:1084A000DD0AF090DE0A68C0C13AD105B9F48091C6
:1084B000DF0A9091E00A892B61F482E090E033D5E5
:1084C00025EB32E0FC01318320839093E00A809316
:1084D000DF0AE090DF0AF090E00A67C0C53BD105F3
:1084E000B9F48091E10A9091E20A892B61F482E06B
:1084F00090E019D52FEB32E0DC012D933C93909363
:10850000E20A8093E10AE090E10AF090E20A4DC0AD
:10851000C63BD105B9F48091E30A9091E40A892B16
:1085200061F482E090E0FFD429EC32E0FC01318379
:1085300020839093E40A8093E30AE090E30AF090AA
:10854000E40A33C0C73BD105B9F48091E50A9091A4
:10855000E60A892B61F482E090E0E5D423ED32E075
:10856000DC012D933C939093E60A8093E50AE0901A
:10857000E50AF090E60A19C0C83BD105B1F4809134
:10858000E70A9091E80A892B61F482E090E0CBD46D
:1085900027EE32E0FC01318320839093E80A809338
:1085A000E70AE090E70AF090E80AE114F10489F4A0
:1085B0008DEF92E00E94A8390E94EB240E94F523DF
:1085C00088E394E00E94963986EC93E00E94963905
:1085D00060C089EF92E00E94A8390E94EB240E94BB
:1085E000F5230E94EB241092270710922607C0E083
:1085F000D0E02196C130D10541F085EF92E00E9494
:10860000A8390E94EB240E94F523D701ED91FC913B
:108610000480F581E02DB801C70119950E94EB2473
:10862000A0902607B0902707209719F3C415D50509
:108630001CF4A114B104E9F68AE89BE00E945F0AE9
:10864000181619062CF48AE89BE00E943D0AF4CF24
:10865000AB2809F483C1DD2009F483C10E94D90845
:108660008091380790913907A0913A07B0913B0764
:108670000197A105B10509F074C10E94EB2421E026
:10868000FC0124876EC10E94A8390E94EB240E943D
:10869000F523C801DDD410925A0B1092590B80912A
:1086A000F30A811171C00E94EB24DC011C968C91AD
:1086B000882309F469C00E949016EC01FC01EA5479
:1086C000FD4F108240960E948A2DCE0187579F4F02
:1086D0000E948A2DCE018E5F9E4F0E948A2D0E949D
:1086E00059187C018C01075C1F4FC1E0D0E0680184
:1086F000B8E3CB1AD108F60180818823D9F08EE443
:1087000094E00E94A83982E594E00E94A839CE0145
:108710000E94EA3A86EC93E00E94A83960E08C2F30
:108720000E94D30D40E050E0BE01C7010E94051732
:10873000D6011C92F80180818823F9F08EE494E040
:108740000E94A83989E694E00E94A839CE010E94CF
:10875000EA3A86EC93E00E94A83961E08C2F0E94EF
:10876000D70E60E08C2F0E94D30D41E050E0BE0197
:10877000C7010E940517D8011C9221960F5F1F4F59
:10878000C533D10509F0B3CF0E94EB24FC018485E9
:108790008093F30AC091F10AD091F20A0E94D9089D
:1087A000DC0112968D919C911397C817D90789F017
:1087B0000E94D908FC01828193819093F20A8093F0
:1087C000F10A0E9490160E94F8110E94D9160E9488
:1087D000A9160E94560F6093ED0A7093EE0A8093DB
:1087E000EF0A9093F00A00915C0B10915D0B2091C1
:1087F0005E0B30915F0B601771078207930708F4D7
:10880000A0C0DC01CB01801B910BA20BB30B8938FC
:108810009341A105B10508F49EC00E94EB24DC0140
:108820001C968C91882319F089E093E002C085E0C2
:1088300093E00E94A8390E94EB240E94F5230E9435
:108840009016EC01FC01E956FD4F8081882341F030
:10885000CE0185589E4F0E9441116B017C0107C0DB
:10886000FE01E35BFF4FC080D180E280F3800E9475
:10887000EB24C092B00AD092B10AE092B20AF09210
:10888000B30AFE01E856FD4F8081882341F0CE01F6
:108890008B569E4F0E9441116B017C0107C0FE0167
:1088A000EA53FF4FC080D180E280F3800E94EB2426
:1088B000C092B40AD092B50AE092B60AF092B70A12
:1088C000FE01E756FD4F8081882341F0CE0181559E
:1088D0009E4F0E9441116B017C0106C0C15CDE4FBE
:1088E000C880D980EA80FB800E94EB24C092B80A3D
:1088F000D092B90AE092BA0AF092BB0A0E94EB2425
:108900000E9448240E9490160E94DA150E94EB24CF
:108910000E9452250E94EB240E9407248091E90ABC
:108920009091EA0AA091EB0AB091EC0A0196A11D80
:10893000B11D8093E90A9093EA0AA093EB0AB093E1
:10894000EC0A0E94560F60935C0B70935D0B809352
:108950005E0B90935F0B0E94FC0AB2C881EF92E01D
:1089600002C08DEE92E00E94A8390E94EB240E9482
:10897000F5230E94EB241092AC0A1092AD0A1092DB
:10898000AE0A1092AF0A85CE0115110509F021CC6F
:10899000E0CB8091270C9091280C5AC310928D0B3C
:1089A00010928C0B88EE93E0A0E0B0E080938E0BE9
:1089B00090938F0BA093900BB093910B8EE493E068
:1089C00090938B0B80938A0B85EC90E09093970BA0
:1089D0008093960B84EC90E09093990B8093980B86
:1089E00080EC90E090939B0B80939A0B81EC90E04D
:1089F00090939D0B80939C0B82EC90E090939F0B47
:108A000080939E0B86EC90E09093A10B8093A00B3B
:108A10001092A30B1092A40B1092A50B1092A60B10
:108A200082E090E080D22EE533E0FC0131832083A8
:108A300090932E0C80932D0C68EC73E087E29CE001
:108A40000E94380D8091BF0C803320F09FEF9093EF
:108A5000C00C11C08093C00C282F30E0F901EE0F3C
:108A6000FF1F2E0F3F1FF901E15DF34F28EB3BE0A5
:108A7000328321838F5F803390F48093C30C282F3F
:108A800030E0F901EE0FFF1F2E0F3F1FF901E15DEE
:108A9000F34F28EB3BE0328321838F5F03C09FEFCE
:108AA0009093C30C8093BF0C0895EE0FFF1F881F97
:108AB0008BBF0790F691E02D19945058BB27AA2739
:108AC00013D00C941C4E0E940E4E38F00E94154E8E
:108AD00020F039F49F3F19F426F40C940B4E0EF459
:108AE000E095E7FB0C94054EE92F0E942D4E58F3BC
:108AF000BA17620773078407950720F079F4A6F583
:108B00000C944F4E0EF4E0950B2EBA2FA02D0B01B6
:108B1000B90190010C01CA01A0011124FF27591BC2
:108B200099F0593F50F4503E68F11A16F040A22FC8
:108B3000232F342F4427585FF3CF46953795279539
:108B4000A795F0405395C9F77EF41F16BA0B620B38
:108B5000730B840BBAF09150A1F0FF0FBB1F661F7F
:108B6000771F881FC2F70EC0BA0F621F731F841FC2
:108B700048F4879577956795B795F7959E3F08F0E8
:108B8000B0CF9395880F08F09927EE0F97958795AA
:108B9000089512D00C941C4E0E94154E58F00E945D
:108BA0000E4E40F029F45F3F29F00C94054E511110
:108BB0000C94504E0C940B4E0E942D4E68F399234A
:108BC000B1F3552391F3951B550BBB27AA276217C9
:108BD0007307840738F09F5F5F4F220F331F441FD6
:108BE000AA1FA9F334D00E2E3AF0E0E831D091500C
:108BF0005040E695001CCAF72AD0FE2F28D0660FF9
:108C0000771F881FBB1F261737074807AB07B0E839
:108C100009F0BB0B802DBF01FF2793585F4F32F047
:108C20009E3F510570F0F1C70C94504E5F3FE4F346
:108C3000983ED4F3869577956795B795F7959F5F9E
:108C4000C9F7880F911D9695879597F90895E1E0EA
:108C5000660F771F881FBB1F621773078407BA0749
:108C600020F0621B730B840BBA0BEE1F88F7E095A4
:108C7000089505D06894B1110C94504E0895F5D71D
:108C800088F09F5790F0B92F9927B751A0F0D1F0F5
:108C9000660F771F881F991F1AF0BA95C9F712C07F
:108CA000B13081F0FCD7B1E00895F9C7672F782F74
:108CB0008827B85F39F0B93FCCF3869577956795EB
:108CC000B395D9F73EF490958095709561957F4F57
:108CD0008F4F9F4F08950FD708F48FEF08950BD74C
:108CE000880B990B08956F927F928F929F92AF920B
:108CF000BF92CF92DF92EF92FF920F931F93CF9389
:108D0000DF93EC01009781F4CB01DF91CF911F91AC
:108D10000F91FF90EF90DF90CF90BF90AF909F901A
:108D20008F907F906F90FFC0FC01E60FF71F9C01B2
:108D300022503109E217F30708F4A8C0D9010D91B8
:108D40001C91119706171707A8F00530110508F4B4
:108D50009BC0C80104978617970708F495C0025076
:108D60001109061B170B019311936D937C93CF018F
:108D70006FD18AC05B01A01AB10A4C01800E911E0E
:108D8000A091CA0CB091CB0C40E050E0E12CF12C4A
:108D9000109709F44AC0A815B905D1F56D907C90DB
:108DA0001197630182E0C80ED11CCA14DB0480F164
:108DB000A3014A195B096A0182E0C80ED11C129610
:108DC000BC9012971396AC91B5E0CB16D10440F04D
:108DD000B282A38351834083D9016D937C930AC0EF
:108DE0000E5F1F4FC301800F911FF9019183808394
:108DF000EB2DFA2FE114F10431F0D7011396FC9317
:108E0000EE93129741C0F093CB0CE093CA0C3CC098
:108E10008D919C9111974817590708F4AC017D0179
:108E200012960D90BC91A02DB3CF8091C80C90915B
:108E3000C90C88159905E1F446175707C8F48091C5
:108E4000020290910302009741F48DB79EB74091C2
:108E5000060250910702841B950BE817F907B0F43E
:108E6000F093C90CE093C80CF901718360830CC0C6
:108E7000CB0159D07C01009749F0A801BE011BD05D
:108E8000CE01E6D0C70104C0CE0102C080E090E070
:108E9000DF91CF911F910F91FF90EF90DF90CF90D6
:108EA000BF90AF909F908F907F906F90089581E0DA
:108EB00090E0F8946EC7FB01DC0102C001900D92B6
:108EC00041505040D8F70895FB01DC018D9101908D
:108ED00080190110D9F3990B0895FB01DC01019071
:108EE0000D920020E1F70895EF920F931F93CF9317
:108EF000DF93E80147FD02C034E001C034E1E42F14
:108F0000440FFF0BF7FF03C0F195E195F109E32E44
:108F1000022F2E2FAE01B3D1CE01DF91CF911F9141
:108F20000F91EF900895CF93DF938230910510F465
:108F300082E090E0E091CA0CF091CB0C20E030E0B0
:108F4000C0E0D0E0309711F14081518148175907B6
:108F5000C0F04817590761F482819381209719F076
:108F60009B838A832BC09093CB0C8093CA0C26C022
:108F70002115310519F04217530718F49A01BE0163
:108F8000DF01EF010280F381E02DDCCF21153105F7
:108F900009F1281B390B2430310590F412968D917C
:108FA0009C9113976115710521F0FB0193838283D6
:108FB00004C09093CB0C8093CA0CFD01329644C040
:108FC000FD01E20FF31F81939193225031092D93FC
:108FD0003C933AC02091C80C3091C90C232B41F42A
:108FE00020910402309105023093C90C2093C80CE3
:108FF00020910202309103022115310541F42DB771
:109000003EB74091060250910702241B350BE091B8
:10901000C80CF091C90CE217F307A0F42E1B3F0B0C
:109020002817390778F0AC014E5F5F4F24173507DA
:1090300048F04E0F5F1F5093C90C4093C80C8193AA
:10904000919302C0E0E0F0E0CF01DF91CF9108956D
:109050000F931F93CF93DF93009709F48CC0FC010B
:109060003297138212820091CA0C1091CB0C011519
:10907000110581F420813181820F931F2091C80C4A
:109080003091C90C2817390779F5F093C90CE09392
:10909000C80C71C0D80140E050E0AE17BF0750F4D3
:1090A00012962D913C911397AD012115310509F1CF
:1090B000D901F3CF9D01DA0133832283608171816D
:1090C000860F971F8217930769F4EC012881398175
:1090D000260F371F2E5F3F4F318320838A819B816C
:1090E00093838283452B29F4F093CB0CE093CA0C35
:1090F00042C01396FC93EE931297ED01499159915A
:109100009E01240F351FE217F30771F480819181CE
:10911000840F951F029611969C938E938281938162
:1091200013969C938E931297E0E0F0E0D80112968C
:109130008D919C911397009719F0F8018C01F6CF4F
:109140008D919C9198012E5F3F4F820F931F20912C
:10915000C80C3091C90C2817390769F4309729F4E5
:109160001092CB0C1092CA0C02C013821282109380
:10917000C90C0093C80CDF91CF911F910F910895F6
:109180006627772709C246EC5CE000C0FA01A1918E
:10919000B081009719F41097E1F0CD01DC01CD0109
:1091A0000D90002011F4C00113C0FB012191222376
:1091B00019F02015D9F7F3CFFB012191201519F4EF
:1091C0001E92119606C02223C1F70D900020A1F730
:1091D000D001FA01A193B0830895BB274A3031F43E
:1091E000992322F4BDE2909581959F4F30C0BB2713
:1091F0002A3051F4992342F4BDE290958095709500
:1092000061957F4F8F4F9F4F01C0BB27FA01A62F5B
:109210006217710581059105330B30FB66F0AA27B3
:10922000660F771F881F991FAA1FA21710F0A21B95
:1092300063953850A9F7A05DAA3308F0A95DA19302
:1092400036F7B111B1931082CA0104C4BB27FB01E8
:109250005527AA27880F991FAA1FA41710F0A41B2F
:1092600083955051B9F7A05DAA3308F0A95DA19389
:10927000009779F7B111B1931192CB01EBC34F92E3
:109280005F926F927F929F92AF92BF92CF92DF9246
:10929000EF92FF920F931F93CF93DF93CDB7DEB77B
:1092A00029970FB6F894DEBF0FBECDBF6A01122F0B
:1092B000B02E2BE3201720F0FF24F394F00E02C011
:1092C000BCE3FB2E0F2D27E0AE014F5F5F4FCAD2EC
:1092D000AC018981982F9970913031F0E1FC06C082
:1092E000E0FE06C090E205C09DE203C09BE201C023
:1092F00090E0EE2DE07183FF3CC0911102C083E04D
:1093000001C084E0811718F4212F281B01C020E040
:10931000E1110BC0F601822F30E2882319F031935E
:109320008150FBCFC20ED11C20E0992329F0D60139
:109330009C93F60131966F01C6010396E2FE0AC0C6
:109340003EE4D6013C9341E411964C93119712965A
:109350003C9306C03EE6F601308341E6418332830A
:10936000FC01322F40E2332309F442C041933150D3
:10937000FACF82FF44C0911102C083E001C084E0B3
:10938000811718F4212F281B01C020E0E1110BC028
:10939000F601822F30E2882319F031938150FBCF00
:1093A000C20ED11C20E0992329F0D6019C93F6012E
:1093B00031966F01C6010396E2FE0BC039E4D60177
:1093C0003C933EE411963C93119736E412963C93FD
:1093D00007C039E6F60130833EE6318336E6328354
:1093E000FC01322F40E2332319F041933150FBCF7F
:1093F000FC01E20FF11D10828EEF9FEFB7C0F1E08C
:10940000911101C0F0E06F2F70E01416150624F4DE
:109410009A012F5F3F4F02C021E030E0260F371F37
:10942000BB2029F06B2D70E06F5F7F4F02C060E0C2
:1094300070E0260F371F612F70E0261737071CF4E6
:10944000121B212F01C020E03E2D387159F4D601A6
:10945000322F60E2332319F06D933150FBCFC20EEF
:10946000D11C20E0FF2331F0D6019C93B6016F5F41
:109470007F4F6B01E1110BC0F601922F30E399236E
:1094800019F031939150FBCFC20ED11C20E09F2DDB
:10949000940F3A81782F7071A72E84FF03C0313367
:1094A00009F49150191624F4993018F098E001C08D
:1094B00091E0E42F852F57FF02C0E0E080E06E2F9F
:1094C000782FE0E0F0E0AEE29A2E3A01691A7108D6
:1094D0002A01461A570A0B2D10E011950195110922
:1094E0006F3F8FEF780729F4D6019C92C601019651
:1094F0006C014617570784F0661677066CF47F01F7
:10950000E40CF51CA1E0B0E0AC0FBD1FEA0EFB1EA1
:10951000D7011196BC9002C090E3B92E6150710939
:109520003196C60101967C016017710724F0D601BF
:10953000BC926C01D5CF6417750741F4363320F423
:10954000353321F4A11002C081E3B82EF601B082B8
:10955000F701822F90E2882319F091938150FBCF7D
:10956000F701E20FF11D108280E090E029960FB61E
:10957000F894DEBF0FBECDBFDF91CF911F910F9149
:10958000FF90EF90DF90CF90BF90AF909F907F9033
:109590006F905F904F9008956F927F928F929F92FD
:1095A000AF92BF92CF92DF92EF92FF920F931F93F1
:1095B000CF93DF93EC017B016115710519F0DB019D
:1095C0008D939C938E010F5F1F4F7880872D90E0C5
:1095D00021D2892B11F0E801F5CFBDE27B1205C045
:1095E0000F5F1F4F7980C1E008C0EBE27E1204C01C
:1095F0008E010E5F1F4F7980C0E06801F1E0CF1A45
:10960000D10843E050E064E174E0C6010BD2892B3D
:10961000E9F4680122E0C20ED11C45E050E06FE0A1
:1096200074E0C601FFD1892B21F4680187E0C80EE0
:10963000D11CE114F10419F0D701CD92DC92C111D3
:10964000F9C060E070E080E89FE7FDC043E050E0D3
:109650006CE074E0C601E6D1892B51F4E114F10409
:1096600009F4EDC00E5F1F4FF70111830083E7C0BF
:10967000680160E070E0CB0100E010E0F601D0EDA1
:10968000D70DDA3050F52C2F2260622E2C2F287047
:10969000C2FF05C0211127C00F5F1F4F24C0222326
:1096A00011F001501109A5E0B0E09B01AC0130D3ED
:1096B0004B015C01880C991CAA1CBB1CC501B401A0
:1096C0006D0F711D811D911D6839A9E97A078A07FF
:1096D000A9E19A0740F0C66005C0DE3F51F4C3FD22
:1096E00044C0C8606C2EBFEFCB1ADB0A7080C62D59
:1096F000C5CF2D2F2F7D2531C1F540814D3211F47D
:10970000C06106C04B3221F0319621E030E006C046
:109710003296D60111964C9122E030E0A0EDA40FD4
:10972000AA3018F0E21BF30B20C040E050E04038B4
:10973000BCE05B075CF49A01220F331F220F331F3A
:10974000420F531F440F551F4A0F511D3196DF0121
:1097500011972C91A0EDA20FAA3048F3C4FF03C0CB
:10976000519541955109040F151FC1FF07C0E11420
:10977000F10421F03197D701ED93FC937FD1C370B1
:10978000C33019F06B017C0106C06B017C01F7FA54
:10979000F094F7F8F09420E030E0A901C701B60199
:1097A00069D1882309F443C017FF06C011950195BC
:1097B0001109CBE2D4E002C0C3E4D4E05E01B8E119
:1097C000AB1AB1084601BE2DAF2D90E2E92EF12C67
:1097D0000E151F057CF0FE012591359145915491A0
:1097E000B4018B2F9A2FABD14B01B82FA92F0E1993
:1097F0001F09EECF2497F594E794CA15DB0541F7CE
:109800006401EB2EFA2E8E2D880F8F2D881F8F3F2F
:1098100041F020E030E0A901C701B6012BD1811150
:1098200006C082E290E09093CD0C8093CC0CC701EF
:10983000B60109C060E070E080E89FEF04C060E01E
:1098400070E080EC9FE7DF91CF911F910F91FF9027
:10985000EF90DF90CF90BF90AF909F908F907F90D0
:109860006F900895283008F027E03327DA01990F28
:10987000311D87FD916000966105710539F43260F4
:109880002E5F3D9330E32A95E1F708959F3F30F036
:1098900080387105610509F03C5F3C5F3D93913074
:1098A00008F08068911DDF93CF931F930F93FF9271
:1098B000EF92192F987F9695E92F96959695E90F37
:1098C000FF27EF55FB4F99273327EE24FF24A701ED
:1098D000E70105900894079428F4360FE71EF81E58
:1098E000491F511D660F771F881F991F0694A1F706
:1098F0000590079428F4E70EF81E491F561FC11D56
:10990000770F881F991F661F0694A1F7059007948B
:1099100028F4F80E491F561FC71FD11D880F991F25
:10992000661F771F0694A1F70590079420F4490F4E
:10993000561FC71FD81F990F661F771F881F0694D1
:10994000A9F784911095177041F0D695C795579552
:109950004795F794E7941A95C1F7E7E4F4E0689423
:109960001590159135916591959105907FE27395CC
:10997000E118F10A430B560BC90BD009C0F7E10CF3
:10998000F11E431F561FC91FD01D7EF4703311F402
:109990008A95E6CFE894015030F0080F0AF40027CA
:1099A000021708F4202F2395022F7A3328F079E349
:1099B0007D932A95E9F710C07D932A9589F6069440
:1099C00097956795379517951794E118F10A430B0A
:1099D000560BC90BD00998F023957E9173957A3375
:1099E00008F070E37C932013B8F77E9170617D934B
:1099F00030F0839571E37D9370E32A95E1F71124AC
:109A0000EF90FF900F911F91CF91DF91992787FDE4
:109A1000909508959111F6C0803219F089508550C3
:109A2000D0F70895FB01DC014150504088F08D9142
:109A300081341CF08B350CF4805E659161341CF030
:109A40006B350CF4605E861B611171F3990B089500
:109A5000881BFCCFDC01FC01672F71917723E1F7B4
:109A6000329704C07C916D9370836291AE17BF07EB
:109A7000C8F3089540D008F481E00895E89409C03F
:109A800097FB3EF490958095709561957F4F8F4F31
:109A90009F4F9923A9F0F92F96E9BB279395F69547
:109AA000879577956795B795F111F8CFFAF4BB0FC5
:109AB00011F460FF1BC06F5F7F4F8F4F9F4F16C029
:109AC000882311F096E911C0772321F09EE8872FB3
:109AD000762F05C0662371F096E8862F70E060E06F
:109AE0002AF09A95660F771F881FDAF7880F9695E8
:109AF000879597F90895990F0008550FAA0BE0E88C
:109B0000FEEF16161706E807F907C0F0121613063F
:109B1000E407F50798F0621B730B840B950B39F47F
:109B20000A2661F0232B242B252B21F408950A26E5
:109B300009F4A140A6958FEF811D811D08950BD0DA
:109B40007BC06CD028F071D018F0952309F05DC06F
:109B500062C01124A5C081D0A0F3959FD1F3950FC9
:109B600050E0551F629FF001729FBB27F00DB11DA1
:109B7000639FAA27F00DB11DAA1F649F6627B00D31
:109B8000A11D661F829F2227B00DA11D621F739F1A
:109B9000B00DA11D621F839FA00D611D221F749F28
:109BA0003327A00D611D231F849F600D211D822F6F
:109BB000762F6A2F11249F5750408AF0E1F08823B6
:109BC0004AF0EE0FFF1FBB1F661F771F881F9150C3
:109BD0005040A9F79E3F510570F017C061C05F3F2C
:109BE000ECF3983EDCF3869577956795B795F795F6
:109BF000E7959F5FC1F7FE2B880F911D969587957E
:109C000097F9089599278827089597F99F6780E81D
:109C100070E060E008959FEF80EC089500240A94BE
:109C20001616170618060906089500240A94121637
:109C30001306140605060895092E0394000C11F46A
:109C4000882352F0BB0F40F4BF2B11F460FF04C017
:109C50006F5F7F4F8F4F9F4F089557FD9058440F70
:109C6000551F59F05F3F71F04795880F97FB991F7B
:109C700061F09F3F79F08795089512161306140638
:109C8000551FF2CF4695F1DF08C0161617061806C5
:109C9000991FF1CF86957105610508940895E894A0
:109CA000BB2766277727CB0197F90895F999FECF4F
:109CB00092BD81BDF89A992780B50895262FF9990C
:109CC000FECF1FBA92BD81BD20BD0FB6F894FA9A9F
:109CD000F99A0FBE01960895052E97FB16F400948D
:109CE0000FD057FD05D024D007FC02D046F408C0A1
:109CF00050954095309521953F4F4F4F5F4F0895B8
:109D000090958095709561957F4F8F4F9F4F0895E7
:109D100031D0A59F900DB49F900DA49F800D911DF3
:109D200011240895B7FFF4CFF3DF821B930B08953E
:109D3000A1E21A2EAA1BBB1BFD010DC0AA1FBB1F4F
:109D4000EE1FFF1FA217B307E407F50720F0A21BC1
:109D5000B30BE40BF50B661F771F881F991F1A942E
:109D600069F760957095809590959B01AC01BD0158
:109D7000CF010895A29FB001B39FC001A39F700DB2
:109D8000811D1124911DB29F700D811D1124911D03
:109D9000089512E0C2EAD2E000E006C0802FFE0182
:109DA0000E9455452196011DC33AD10780E008075E
:069DB000A9F7F894FFCFB3
:109DB600FFFF0000CE0C800001000000200A0D000D
:109DC60000000000000B0A18072607000000000A22
:109DD6000A16075A0900000000AE23BB214C2500D5
:109DE600000000AD23B921712300000000AC23B7A9
:109DF60021402300000000AB23B5210F2300000003
:109E060000AA23B321D62200000000A923B1219D78
:109E16002200000000A823AF21642200000000A752
:109E260023AD21282500000000A623AB21F3210045
:109E3600000000A523A921022200000000A423A7F8
:109E460021482100000000A323A321D42100000003
:109E560000A223A521BD2100000000110A240765E8
:109E66002100000000100A22071B08000000000F56
:109E76000A2007EC07000000000E0A1E07E507008F
:109E86000000000D0A1C07030700000000090A1461
:109E960007A206000000000C0A1A077C075230339E
:109EA60000523032005230370052303100523039D1
:109EB60000523837005230300052383700523038AE
:109EC60000362E302E312E52000001000000010017
:109ED600000001000000523835005238340052307C
:109EE6003500523036005231330052313200523191
:109EF6003100523837005230340000000000950A15
:109F0600120A5F0A3D0A510ADB0A00000000080A2D
:109F1600120752393920484F4D45205A204F4E20BE
:109F2600535441525455500D0A0052393920484F66
:109F36004D452059204F4E20535441525455500DF3
:109F46000A0052393920484F4D452058204F4E209F
:109F5600535441525455500D0A005239392041523A
:109F66004455494E4F205354415254555020434F67
:109F76004D504C4554450D0A002A004730004730E5
:109F8600300047310047303100473238004630391B
:109F96000046390046313100463132004631330041
:109FA60046313400463135004631360046323000FF
:109FB60046323100463232004633310046333200F3
:109FC60046343100463432004634330046343400D9
:109FD60046363100463831004638320046383300BE
:109FE60046383400200A0D005239392068616E6403
:109FF6006C6572203D3D204E554C4C0D0A00523981
:10A00600390020726573657474696E6720646967C8
:10A016006974616C2070696E002072657365747472
:10A02600696E6720616E616C6F672070696E0052A1
:10A03600383320005239392057696C6C207A6572A2
:10A046006F2058005239392057696C6C207A657236
:10A056006F2059005239392057696C6C207A657225
:10A066006F205A00686F6D650D0A0052323100503C
:10A07600005600523939204572726F723A20696E65
:10A0860076616C696420706172616D6574657220B9
:10A0960069640D0A005234310052393920656D6504
:10A0A6007267656E63792073746F700D0A0052399A
:10A0B60039206572726F720D0A00523832005239B9
:10A0C600392073746F707065640D0A005239392037
:10A0D6006572726F722000206465616374697661CF
:10A0E6007465206D6F746F722058206475652074D6
:10A0F6006F206D69737365642073746570730020D7
:10A1060064656163746976617465206D6F746F72DE
:10A1160020592064756520746F206D6973736564BA
:10A126002073746570730020646561637469766179
:10A136007465206D6F746F72205A20647565207483
:10A146006F206D6973736564207374657073005254
:10A1560039392074696D656F757420582061786986
:10A16600730D0A005239392074696D656F75742054
:10A176005920617869730D0A005239392074696D66
:10A18600656F7574205A20617869730D0A00205135
:10A1960000523831002058410020584200205941D1
:10A1A6000020594200205A4100205A4200523230C3
:10A1B6000020737461200020637572200020656E94
:10A1C6006420002068616C662000206C656E2000AB
:10A1D600206D696E2000206D617820002073706408
:10A1E60020005239392043616C6962726174696F6B
:10A1F6006E206572726F723A20696E76616C696460
:10A2060020617869732073656C65637465640D0AF3
:10A216000020617869732000206174207374617274
:10A2260074696E6720706F696E7400523233002055
:10A2360063616C6962726174696E67206C656E67D2
:10A24600746800207374657020636F756E743A20AD
:10A2560000523939206D6F76656D656E7420646FB6
:10A266006E650D0A0020617420656E6420706F694A
:10A276006E74005239392043616C69627261746987
:10A286006F6E206572726F723A20656E6420737409
:10A296006F7020616374697665206265666F7265AA
:10A2A6002073746172740D0A00206D6F76652074D8
:10A2B6006F20737461727420666F722063616C69BB
:10A2C60062726174696F6E006E616E00696E66001F
:04A2D6006F76660039
:00000001FF
